:1062DB00E5467006127AED8F4622E546B4050612A6
:1062EB003B758F4622E546B40B061270FA8F462299
:1062FB00E546B40A061268368F4622E546B40F0609
:10630B001270668F4622E546B414061264E78F4678
:10631B0022E546B41906127A308F4622E546B41EA2
:10632B0006127B018F4622E546B42306126C438F7F
:10633B004622E546B42806127BB68F4622E546B4C4
:10634B002D06127B158F4622E546B4320512739E3D
:03635B008F462248
:107AED00C20890061EE0FFA3E0901CECCFF0A3EFC0
:047AFD00F07F0522EF
:103B7500127BB250477D047F011262535008E53E27
:103B8500B401037F0B227D047F021262535008E5C6
:103B95003EB402037F0B227D047F0312625350085B
:103BA500E53EB403037F0B227D047F04126253506C
:103BB50008E53EB404037F0B227F0A227F081275B5
:103BC5004D500612534B7F00227D057F051262532F
:103BD5005032901CEEE07002A3E070282046257D4F
:103BE500017F011262534003023CEB90066CE0FF3B
:103BF5007C0A7D701272E3900610E0FFA3E0901C32
:103C0500EE023CB27D067F051262535031901CF0E6
:103C1500E07002A3E070272048247D017F02126234
:103C2500534003023CEB90066DE0FF7C0A7D901249
:103C350072E3900612E0FFA3E0901CF0806F7D0711
:103C45007F051262535031901CF2E07002A3E070C0
:103C550027204C247D017F031262534003023CEB75
:103C650090066EE0FF7C0A7DB01272E3900614E0C8
:103C7500FFA3E0901CF280357D087F05126253504A
:103C850033901CF4E07002A3E07029204F267D01DB
:103C95007F04126253504F90066FE0FF7C0A7DD07F
:103CA5001272E3900616E0FFA3E0901CF4CFF0A398
:103CB500EFF080327D077F06126253500F30290CDA
:103CC500901CECE07002A3E07002C22930380C9021
:103CD5001CECE07002A3E07002C238786CE6B40513
:093CE500057F04125D9F7F05229A
:1070FA00203842900633E0901D10F0123346E53EE8
:10710A00B401062049247F0522E53EB40206204D3B
:10711A00197F0522E53EB4030620510E7F0522E5BC
:10712A003EB404062054037F0522901D10E0D39438
:08713A000050C8D2387F0A2280
:10683600E53B700AE53EB40105753B018028E53B62
:10684600700AE53EB40205753B02801AE53B700A04
:10685600E53EB40305753B03800CE53B7008E53E59
:10686600B40403753B047D077F06126253500C7D0A
:10687600077F06126253501E30291B900650E0FF18
:106886007C067DF01272E37D017F01126253500691
:09689600120FB3122B647F0F22D4
:10706600127BB2503F120FB3202F09203006203179
:1070760003303209E5327005127742800B786CE6F0
:10708600B4050B7F03125D9F122B64120FB3202FE2
:107096001020300D20310A203207E5327003122B02
:0A70A600647F0F221277427F14224C
:1064E700E4F53B7D077F06126253500C7D077F065C
:1064F700126253505E30295B786CE670047F01802E
:1065070008786CE6B404077F02125D9F8038786CC8
:10651700E6B407047601802E7D037F05126253508F
:1065270025901CF6E07002A3E0701B900662E0FF66
:106537007C097D301272E3900620E0FFA3E0901CF7
:10654700F6CFF0A3EFF07F0612754D50037F0022C0
:106557007F19227D077F0612625350052029027F8B
:0265670005220B
:107A30007D077F0612625350062029037F0522909E
:0A7A40000630E0901D10F07F1E22BA
:107B0100901D10E070037F2322127BB250037F0A85
:047B1100227F1E228F
:106C43007D047F071262535041E53EB4010B900669
:106C53005EE0FF7C087DB0802EE53EB4020B90061B
:106C63005FE0FF7C087DD0801EE53EB4030B9006F9
:106C730060E0FF7C087DF0800EE53EB4040C9006D6
:106C830061E0FF7C097D101272E3900631E0901DF4
:056C930010F07F282233
:037BB6007F2D22FE
:107B1500901D10E070037F3222127BB250037F0A62
:047B2500227F2D226C
:10739E003058037F32227D047F05126253502890AD
:1073AE001CF8E07002A3E0701E900663E0FF7C09FB
:1073BE007D501272E3900622E0FFA3E0901CF8CFFE
:0C73CE00F0A3EFF07F3222C2087F002203
:10721800900640E06038D259D224753D0320692A8F
:10722800123346122B64120FB3127BB25009E53D9C
:10723800600512334680F2E4F522F523127BB24052
:1072480009E53D600512334680F2E53D70CFC2592D
:05725800C224C258220F
:04000E0001000330BA
:0300030002696728
:0B696700C0E0C083C082C0D075D00823
:10697200853082852F83E493FF204404C4540FFFA3
:10698200430FF08F80C284D28500C2870000D28775
:10699200007580FF7580FEC284C28500C287000038
:1069A2000000D287007580FF30440CC2440530E5F8
:0B69B200307006052F8002D244D2A8EE
:0969BD00D0D0D082D083D0E032AA
:03000B00021BB61F
:101BB600C0E0C0F0C083C082C0D075D008758CD894
:101BC600758A92D28C1242221274B2E531D39400F5
:101BD60040051531021F40753111901D10E0D39458
:101BE600004003E014F0901D11E0D394004003E0A0
:101BF60014F0901D12E0D394004003E014F0901D01
:101C060013E0D394004003E014F0E532D39400408F
:101C16000215321541E541B40A004003021F3D900A
:101C26001C2CF8282873021F40021E91021E59021E
:101C36001E2C021DC2021D58021CEE021C84021C30
:101C460067021C4AD3901CEDE09400901CECE094D3
:101C5600005003021F40A3E024FFF0901CEC021F7B
:101C660031D3901CE9E09400901CE8E09400500306
:101C7600021F40A3E024FFF0901CE8021F317F0101
:101C860012780A4003021F40901CE1E09400901C69
:101C9600E0E09400400CA3E024FFF0901CE0E03468
:101CA600FFF0D3901CEFE09400901CEEE09400400F
:101CB6000CA3E024FFF0901CEEE034FFF0D3901C60
:101CC600FBE09400901CFAE094005003021F407D54
:101CD600067F011262534003021F40901CFBE02462
:101CE600FFF0901CFA021F317F0212780A400302AD
:101CF6001F40901CE3E09400901CE2E09400400C2E
:101D0600A3E024FFF0901CE2E034FFF0D3901CF136
:101D1600E09400901CF0E09400400CA3E024FFF057
:101D2600901CF0E034FFF0D3901CFDE09400901C72
:101D3600FCE094005003021F407D067F02126253AE
:101D46004003021F40901CFDE024FFF0901CFC02A3
:101D56001F317F0312780A4003021F40901CE5E002
:101D66009400901CE4E09400400CA3E024FFF09063
:101D76001CE4E034FFF0D3901CF3E09400901CF2D6
:101D8600E09400400CA3E024FFF0901CF2E034FF46
:101D9600F0D3901CFFE09400901CFEE094005003EA
:101DA600021F407D067F031262534003021F4090CC
:101DB6001CFFE024FFF0901CFE021F317F04127806
:101DC6000A4003021F40901CE7E09400901CE6E0E6
:101DD6009400400CA3E024FFF0901CE6E034FFF0F2
:101DE600D3901CF5E09400901CF4E09400400CA302
:101DF600E024FFF0901CF4E034FFF0D3901D01E0E6
:101E06009400901D00E094005003021F407D067F61
:101E1600041262534003021F40901D01E024FFF0AC
:101E2600901D00021F31D3901CEBE09400901CEA39
:101E3600E09400400CA3E024FFF0901CEAE034FF9D
:101E4600F0901D14E0D394005003021F40E014F0FC
:101E5600021F40D3901CF9E09400901CF8E0940017
:101E6600400CA3E024FFF0901CF8E034FFF0D39080
:101E76001CF7E09400901CF6E094005003021F400B
:101E8600A3E024FFF0901CF6021F31786CE6FF7089
:101E960003021F40EFB401059006188027786CE610
:101EA600FFB40219D3901CEBE09400901CEAE09476
:101EB60000403FA3E024FFF0901CEA806EEFB403DD
:101EC6001190061AE0FFA3E0901CEACFF0A3EFF012
:101ED6008020786CE6FFB4041ED3901CEBE09400DF
:101EE600901CEAE09400400AA3E024FFF0901CEA6C
:101EF6008039786C068043EF6405603E786CE6FFB7
:101F0600B4060D901CEA7402F0A37458F006802AF9
:101F1600EFB40726D3901CEBE09400901CEAE09403
:101F260000400EA3E024FFF0901CEAE034FFF080AE
:101F360009786C7600800375410A1279DD40081233
:101F4600761040031279F9D0D0D082D083D0F0D069
:021F5600E03277
:0300130002613B4C
:0D613B00C0E0C0F0C083C082C0D075D0109D
:1061480075A0FFC284C285D287C286308018C2A4D7
:10615800C2A5D2A6C2A7E5A0540FF54AD2A7FF123E
:1061680065E9D286804F308118D2A4C2A5D2A6C2D2
:10617800A7E5A0540FF54AD2A7FF12635ED2868026
:1061880034308218C2A4D2A5D2A6C2A7E5A0540F63
:10619800F54AD2A7FF1263E1D2868019308316D25E
:1061A800A4D2A5D2A6C2A7E5A0540FF54AD2A7FF4C
:0561B800126464D286B0
:0B61BD00D0D0D082D083D0F0D0E032F0
:106BEC00BF0113900632E0901D10F0901D10E0D301
:106BFC009400404280F5BF0213900632E0901D11C4
:106C0C00F0901D11E0D39400402C80F5BF0313903D
:106C1C000632E0901D12F0901D12E0D39400401645
:106C2C0080F5BF0411900632E0901D13F0901D13F7
:076C3C00E0D3940050F722A1
:106C9800304712205F0F900672E0FF7C0B7D3012A8
:106CA80072E3D25F22304B1220610F900673E0FF2F
:106CB8007C0B7D501272E3D26122304E1220620F9B
:106CC800900674E0FF7C0B7D701272E3D262223072
:106CD800521120630E900675E0FF7C0B7D901272B6
:046CE800E3D263226E
:1055CB00303D1A204617900664E0FF7C097D70126F
:1055DB0072E3D246C214C210C21CC2182230461447
:1055EB00203911900665E0FF7C097D901272E3C2B1
:1055FB0046C23D22303E1A204817900666E0FF7CDB
:10560B00097DB01272E3D248C215C211C21DC21974
:10561B0022304814203A11900667E0FF7C097DD0B8
:10562B001272E3C248C23E2230401A204C17900639
:10563B0068E0FF7C097DF01272E3D24CC216C212F5
:10564B00C21EC21A22304C14203B11900669E0FF97
:10565B007C0A7D101272E3C24CC2402230421A20E7
:10566B004F1790066AE0FF7C0A7D301272E3D24F2F
:10567B00C217C213C21FC21B22304F13203C109003
:10568B00066BE0FF7C0A7D501272E3C24FC24222CE
:10518000124108D28C7F0712754D5005120016800F
:105190001212718A7F1F7E0012783190001FEFF08B
:1051A00012766A7F0812754D500512599480FE9050
:1051B00006087402F0A37458F090060A7402F0A373
:1051C0007458F090060C7402F0A37458F090060E18
:1051D0007402F0A37458F0900681E0FF7C0D7D10FE
:1051E0001272E3E4FFEFFD3395E0FC74302DF5829D
:1051F00074003CF583E0FE74F02DF582741A3CF5E2
:1052000083EEF00FBF08DED2081279F97545017FF1
:1052100001125D9F900618E0FFA3E0901CEACFF01A
:10522000A3EFF0C2081279F9123346305A11E53E65
:10523000B4010C900651E0FF7C077D101272E3125E
:1052400062DB305B0312444D305C0312433A305D45
:105250000312489030600312499A124DA97D077FCE
:10526000061262534002C2291255CB126C9880B8C4
:10444D007C007D80C2677F011236B950117F061244
:10445D00754D5002D2087F01121F580244ED7C00A9
:10446D007D70D2677F011236B95002800D7C007DC0
:10447D0078D2677F011236B950077F01120941804A
:10448D005F7C007DA0D2677F011236B950117D0788
:10449D007F06126253500875450112776B80417C7F
:1044AD00007DA8C2677F011236B950197D057F01C5
:1044BD0012625350107F0612754D5002D2087F01C3
:1044CD0012455F801B7C007DB0C2677F011236B93B
:1044DD00500E7F0612754D5002D2087F01124F9972
:1044ED00E4F54CAF4CEF3395E0FEEF7803C333CEDC
:1044FD0033CED8F92400F58274013EAD82FCD2672B
:10450D007F011236B95038754501AF4CEF3395E048
:10451D00FE74A02FF58274063EF583E0FFC007AF51
:10452D004CEF3395E0FEEF7805C333CE33CED8F99B
:10453D0024F0F58274103EAD82FCD007126EE105B9
:10454D004CC3E54C648094A84099C25BC265126C63
:01455D00EC71
:01455E00223A
:10433A007F0612754D5002C2087D017F0612625334
:10434A00503D7C007D88C2677F021236B9500BD27D
:10435A00097F02121F58C20980257C007D70D2672E
:10436A007F021236B95002800D7C007D78D2677FB9
:10437A00021236B95009D2097F02120941C20990C4
:10438A00001FE030E1427C007DA0D2677F02123636
:10439A00B950147D077F06126253500B1278577575
:1043AA00450212776B801E7C007DA8C2677F0212CD
:1043BA0036B950147D057F02126253500B1278579A
:1043CA007F0212455F1279487D027F0612625350BE
:1043DA006AE4F54CAF4CEF3395E0FEEF7803C33354
:1043EA00CE33CED8F92400F58274013EAD82FCD2D8
:1043FA00677F021236B95038754502AF4CEF3395D4
:10440A00E0FE74A02FF58274063EF583E0FFC00734
:10441A00AF4CEF3395E0FEEF7805C333CE33CED8F9
:10442A00F924F0F58274103EAD82FCD007126EE1D9
:10443A00054CC3E54C648094A84099C25CC26612DC
:02444A006D40C3
:01444C00224D
:104890007D037F06126253503D7C007D90C2677F8E
:1048A000031236B9500BD20E7F03121F58C20E806E
:1048B000257C007D70D2677F031236B95002800DCF
:1048C0007C007D78D2677F031236B95009D20E7F03
:1048D00003120941C20E90001FE030E2427C007DCD
:1048E000A0D2677F031236B950147D077F0612628B
:1048F00053500B12785775450312776B801E7C005E
:104900007DA8C2677F031236B950147D057F03125C
:104910006253500B1278577F0312455F1279487D1E
:10492000047F06126253506AE4F54CAF4CEF3395A6
:10493000E0FEEF7803C333CE33CED8F92400F582FE
:1049400074013EAD82FCD2677F031236B9503875D0
:104950004503AF4CEF3395E0FE74A02FF58274064B
:104960003EF583E0FFC007AF4CEF3395E0FEEF78F4
:1049700005C333CE33CED8F924F0F58274103EADA2
:1049800082FCD007126EE1054CC3E54C648094A80C
:094990004099C25DC228126D9429
:0149990022FB
:10499A007D057F06126253503D7C007D98C2677F79
:1049AA00041236B9500BD20C7F04121F58C20C8065
:1049BA00257C007D70D2677F041236B95002800DC3
:1049CA007C007D78D2677F041236B95009D20C7FF9
:1049DA0004120941C20C90001FE030E3427C007DC2
:1049EA00A0D2677F041236B950147D077F0612627F
:1049FA0053500B12785775450412776B801E7C0052
:104A0A007DA8C2677F041236B950147D057F04124F
:104A1A006253500B1278577F0412455F1279487D12
:104A2A00067F06126253506AE4F54CAF4CEF339599
:104A3A00E0FEEF7803C333CE33CED8F92400F582F3
:104A4A0074013EAD82FCD2677F041236B9503875C4
:104A5A004504AF4CEF3395E0FE74A02FF58274063F
:104A6A003EF583E0FFC007AF4CEF3395E0FEEF78E9
:104A7A0005C333CE33CED8F924F0F58274103EAD97
:104A8A0082FCD007126EE1054CC3E54C648094A801
:094A9A004099C260C22A126DE8C5
:014AA30022F0
:106F8100BF010AC214C210C21CC2188025BF020A66
:106F9100C215C211C21DC2198018BF030AC216C28E
:106FA10012C21EC21A800BBF0408C217C213C21F2D
:106FB100C21B90001FE0FF30E002D224EF30E1025B
:0E6FC100D225EF30E202D226EF30E302D227D3
:016FCF00229F
:1065E9008F4B7868E6C39450507130496E20596BCF
:1065F9007D077F01126253502B205E287868E67070
:106609000D90063BE0B54B06203F03D23F22202FD9
:106619000D203F0A7F01126F81753D02D22F90062E
:1066290034E0F5327D087F06126253501990063F17
:10663900E0B54B06205E03D265220534E534AE335E
:10664900700E0533800A0534E534AE337002053324
:0C66590014F5828E83E54BF07868062271
:10635E008F4B7869E6C394505078304D7520597242
:10636E007D077F0212625350327F0212780A502B41
:10637E00205E287869E6700D90063BE0B54B06204E
:10638E004103D2412220300D20410A7F02126F813B
:10639E00753D02D230900634E0F5327D087F06124C
:1063AE006253501990063FE0B54B06205E03D2664D
:1063BE00220536E536AE35700E0535800A0536E512
:1063CE0036AE357002053514F5828E83E54BF078C6
:0363DE006906222B
:1063E1008F4B786AE6C394505078305175205972BA
:1063F1007D077F0312625350327F0312780A502BBC
:10640100205E28786AE6700D90063BE0B54B0620C9
:106411004303D2432220310D20430A7F03126F81AF
:10642100753D02D231900634E0F5327D087F0612C7
:106431006253501990063FE0B54B06205E03D22807
:10644100220538E538AE37700E0537800A0538E584
:1064510038AE377002053714F5828E83E54BF0783C
:036461006A0622A6
:106464008F4B786BE6C39450507830547520597232
:106474007D077F0412625350327F0412780A502B36
:10648400205E28786BE6700D90063BE0B54B062045
:106494004503D2452220320D20450A7F04126F8124
:1064A400753D02D232900634E0F5327D087F061243
:1064B4006253501990063FE0B54B06205E03D22A82
:1064C40022053AE53AAE39700E0539800A053AE5F7
:1064D4003AAE397002053914F5828E83E54BF078B3
:0364E4006B062222
:1078570090001FE0FF30E004D208D220EF30E104AF
:10786700D209D221EF30E204D20ED222EF30E30464
:05787700D20CD2232217
:10794800C220C221C222C22390001FE0FF30E10200
:0F795800C209EF30E202C20EEF30E302C20C228E
:105D9F008F4C304603025E3B304803025E3B304C73
:105DAF0003025E3B304F03025E3B7D017F011262B7
:105DBF00535079E54CB401197D017F0512625350A0
:105DCF000C90065AE0FF7C087D301272E3786C0667
:105DDF0022E54CB402177D027F05126253504890A2
:105DEF00065BE0FF7C087D501272E3803AE54CB40D
:105DFF00041A7D027F05126253500C90065DE0FF7E
:105E0F007C087D901272E3786C760622E54C640371
:105E1F00701E7D027F05126253500C90065CE0FFEE
:105E2F007C087D701272E3786C760122E4786CF650
:015E3F002240
:107A1500EF1FAA0670011ED39400EA9400400BE400
:0A7A2500FDEDC394C850E90D80F791
:017A2F002234
:105A49008F5D306B5BE55DB40111D22090001FE0E2
:105A5900F420E003305E44D2088040E55DB40211D1
:105A6900D22190001FE0F420E103305E2ED209809C
:105A79002AE55DB40311D22290001FE0F420E2036D
:105A8900305E18D20E8014E55DB4040FD223900065
:105A99001FE0F420E303305E02D20CAF5D026BEC31
:105AA900E55DB40110C22090001FE0F420E003304E
:105AB9005E41C20822E55DB40210C22190001FE0D8
:105AC900F420E103305E2CC20922E55DB40310C263
:105AD9002290001FE0F420E203305E17C20E22E597
:105AE9005DB4040FC22390001FE0F420E303305E8D
:045AF90002C20C22B7
:105AFD008F5330695BE553B40111D22490001FE040
:105B0D00F420E003305E44D2088040E553B4021126
:105B1D00D22590001FE0F420E103305E2ED20980E3
:105B2D002AE553B40311D22690001FE0F420E203BE
:105B3D00305E18D20E8014E553B4040FD2279000B6
:105B4D001FE0F420E303305E02D20CAF53026BEC86
:105B5D00E553B40110C22490001FE0F420E003309F
:105B6D005E41C20822E553B40210C22590001FE029
:105B7D00F420E103305E2CC20922E553B40310C2B8
:105B8D002690001FE0F420E203305E17C20E22E5DE
:105B9D0053B4040FC22790001FE0F420E303305EDE
:045BAD0002C20C2202
:08290E008F538C548D558B563C
:10291600C267E55524FFF582E55434FFF583E0F5FB
:1029260058855582855483E0FFF559A3E0FEF55A94
:10293600EF14B40800505C90294B75F003A4C583CE
:1029460025F0C5837302296302296A0229710229C7
:102956007802297F02298602298D0229947557015A
:10296600D267802F755702D2678028755704D267C1
:102976008021755708D267801A755710D267801361
:10298600755720D267800C755740D26780057557FA
:1029960080D267EE24FE7003022A5B24F8605C2472
:1029A600096003022A6DE553B401059000208045B5
:1029B600E553B40205900021803BE553B40305902E
:1029C60000228031E553B404059000238027E553A7
:1029D600B40505900024801DE553B4060590002536
:1029E6008013E553B407059000268009E553640873
:1029F6007077900027E04557F0806EE553B40105E7
:102A06009000208045E553B40205900021803BE507
:102A160053B403059000228031E553B404059000B9
:102A2600238027E553B40505900024801DE553B4A3
:102A360006059000258013E553B40705900026800F
:102A460009E55364087022900027E0FFE557F4FE7D
:102A5600EF5EF08014E553B4080D855582855483E6
:102A6600E0FF1260A7C267C267206703022B63E517
:102A760053B40109900020E0FD7F208060E553B447
:102A86000209900021E0FD7F218052E553B403093D
:102A9600900022E0FD7F228044E553B404099000B3
:102AA60023E0FD7F238036E553B40509900024E03A
:102AB600FD7F248028E553B40609900025E0FD7FBC
:102AC60025801AE553B40709900026E0FD7F26808D
:102AD6000CE553B4080C900027E0FD7F277E00121A
:102AE6007323D2AFD26BAF56125A49AD58E4FF12D8
:102AF60076EEAD59E4FF1276EEE55AB401047D3860
:102B06008007E55AB40A077D367F061276EEE5534E
:102B1600B4080312766A7D077F06126253500B20B3
:102B26002908C208C209C20EC20C7D017F011262C9
:102B3600534002C2087D017F021262534002C2095D
:102B46007D017F031262534002C20E7D017F041293
:0D2B560062534002C20CC26BAF56125A49C6
:012B6300224F
:045E40008F538D549B
:105E4400D26BAF54125A49AF54126BECE553B40100
:105E5400059000208044E553B40205900021803A67
:105E6400E553B403059000228030E553B404059053
:105E740000238026E553B40505900024801CE553D7
:105E8400B406059000258012E553B407059000265A
:105E94008008E553B40806900027E0F555E5556001
:105EA40025755701E4F556E55530E007AD57E4FF95
:105EB4001276EEE555C313F55505570556E556C359
:105EC400940840E3800E7D187F021276EE7D537FA6
:0B5ED400021276EEC26BAF54125A4966
:015EDF0022A0
:021F58008F4DAB
:101F5A00E54D6401701E754E1B754F10900080E0B0
:101F6A00F550E54F2550F582E4354EF583E0F552FC
:101F7A0078688069E54D6402701E754E1B754F6066
:101F8A00900088E0F550E54F2550F582E4354EF58E
:101F9A0083E0F55278698045E54D6403701E754EFD
:101FAA001B754FB0900090E0F550E54F2550F58233
:101FBA00E4354EF583E0F552786A8021E54DB404A4
:101FCA001F754E1C754F00900098E0F550E54F259F
:101FDA0050F582E4354EF583E0F552786BE6F5511B
:101FEA00E55214B4090040030222F790200375F069
:101FFA0003A4C58325F0C5837302201E0220710243
:10200A0020C402211702216A0221BD0222100222E3
:10201A00610222B1E54F2550F582E4354EF583A3DE
:10202A00E0B40A18E5502402FFE433FEE551B5078F
:10203A000BE4B50607AD4D7F01022286AF507E0044
:10204A00EF2403FDEE33FCE5516D7001EC600302F1
:10205A0022F7EF254FFFEE354ECF2401FDE43FFC7A
:10206A00AB4D7F010222AEE54F2550F582E4354E95
:10207A00F583A3E0B40A18E5502402FFE433FEE531
:10208A0051B5070BE4B50607AD4D7F02022286AFB4
:10209A00507E00EF2403FDEE33FCE5516D7001EC38
:1020AA0060030222F7EF254FFFEE354ECF2401FDE4
:1020BA00E43FFCAB4D7F020222AEE54F2550F5828C
:1020CA00E4354EF583A3E0B40A18E5502402FFE490
:1020DA0033FEE551B5070BE4B50607AD4D7F0302A4
:1020EA002286AF507E00EF2403FDEE33FCE5516DEE
:1020FA007001EC60030222F7EF254FFFEE354ECF59
:10210A002401FDE43FFCAB4D7F030222AEE54F25DF
:10211A0050F582E4354EF583A3E0B40A18E550245D
:10212A0002FFE433FEE551B5070BE4B50607AD4DF2
:10213A007F04022286AF507E00EF2403FDEE33FCBB
:10214A00E5516D7001EC60030222F7EF254FFFEEB7
:10215A00354ECF2401FDE43FFCAB4D7F040222AE95
:10216A00E54F2550F582E4354EF583A3E0B40A180D
:10217A00E5502402FFE433FEE551B5070BE4B5064A
:10218A0007AD4D7F05022286AF507E00EF2403FD86
:10219A00EE33FCE5516D7001EC60030222F7EF2586
:1021AA004FFFEE354ECF2401FDE43FFCAB4D7F05DA
:1021BA000222AEE54F2550F582E4354EF583A3E0C1
:1021CA00B40A18E5502402FFE433FEE551B5070BC3
:1021DA00E4B50607AD4D7F06022286AF507E00EFBA
:1021EA002403FDEE33FCE5516D7001EC600302221D
:1021FA00F7EF254FFFEE354ECF2401FDE43FFCAB50
:10220A004D7F060222AEE54F2550F582E4354EF5A4
:10221A0083A3E0B40A17E5502402FFE433FEE55134
:10222A00B5070AE4B50606AD4D7F07804FAF507E6D
:10223A0000EF2403FDEE33FCE5516D7001EC600301
:10224A000222F7EF254FFFEE354ECF2401FDE43F82
:10225A00FCAB4D7F07804DE54F2550F582E4354EA6
:10226A00F583A3E0B40A18E5502402FFE433FEE53F
:10227A0051B5070BE4B50607AD4D7F08025E40AFC6
:10228A00507E00EF2403FDEE33FCE5516D7001EC46
:10229A00705BEF254FFFEE354ECF2401FDE43FFC86
:1022AA00AB4D7F0802290EE54F2550F582E4354EE5
:1022BA00F583A3A3E07036E54F2550F582E4354E49
:1022CA00F583A3E024F96008147022AF4D0277E386
:1022DA00D26B7F01125A49AF4D126BEC7D5E7F02C1
:0D22EA001276EEC26B7F01125A4912599410
:0122F70022C4
:0436B9008C4D8D4E59
:1036BD00054EE54E7002054D14F5828C83E0F970D0
:1036CD000302385BBF010875331B753410801FBFB3
:1036DD00020875351B7536608014BF030875371BDE
:1036ED007538B08009BF040675391C753A0020671E
:1036FD00030237C1BF01087868E6696002C322BFC3
:10370D0002087869E6696002C322BF0308786AE699
:10371D00696002C322BF0408786BE6696002C322A8
:10372D00E4FEEEC39940030237BFEF6401701CE560
:10373D004E2EF582E4354DF583E0FDE5342EF58210
:10374D00E43533F583E06D6002C322EF6402701C33
:10375D00E54E2EF582E4354DF583E0FDE5362EF58B
:10376D0082E43535F583E06D6002C322EF640370AA
:10377D001CE54E2EF582E4354DF583E0FDE5382E42
:10378D00F582E43537F583E06D6002C322EF640402
:10379D00701CE54E2EF582E4354DF583E0FDE53ADE
:1037AD002EF582E43539F583E06D6002C3220E02F9
:1037BD00372FD32230670302385CE4FEEEC3994005
:1037CD0003023859EF6401701CE54E2EF582E43585
:1037DD004DF583E0FDE5342EF582E43533F583E0D8
:1037ED006D6065C322EF6402701CE54E2EF582E418
:1037FD00354DF583E0FDE5362EF582E43535F5835F
:10380D00E06D6044C322EF6403701CE54E2EF5821B
:10381D00E4354DF583E0FDE5382EF582E43537F5D9
:10382D0083E06D6023C322EF6404701CE54E2EF51A
:10383D0082E4354DF583E0FDE53A2EF582E4353928
:0F384D00F583E06D6002C3220E0237C9D322C398
:01385C002249
:102B640090001FE0540FF55CB4010BE53EB4010383
:102B7400D21422C21422E55C6403702AE53EB40137
:102B840006D214D2108004C214C210E53EB402115D
:102B9400D2157D017F071262534003022D7FD211AB
:102BA40022C215C21122E55C6405702AE53EB40117
:102BB40006D214D21C8004C214C21CE53EB4031114
:102BC400D2167D027F071262534003022D7FD21E6C
:102BD40022C216C21E22E55C6409702AE53EB401D5
:102BE40006D214D2188004C214C218E53EB40411EB
:102BF400D2177D037F071262534003022D7FD21B3D
:102C040022C217C21B22E55C6407704EE53EB40184
:102C140008D214D210D21C8006C214C210C21CE501
:102C24003EB40211D2157D017F071262535002D2C5
:102C340011D21D8006C215C211C21DE53EB4031394
:102C4400D216D2127D027F071262534003022D7FF7
:102C5400D21E22C216C212C21E22E55C640B704E42
:102C6400E53EB40108D214D210D2188006C214C2B0
:102C740010C218E53EB40211D2157D017F0712621D
:102C8400535002D211D2198006C215C211C219E5DD
:102C94003EB40413D217D2137D037F07126253404C
:102CA40003022D7FD21B22C217C213C21B22E55C72
:102CB400640D704BE53EB40108D214D21CD21880C6
:102CC40006C214C21CC218E53EB40311D2167D021A
:102CD4007F071262535002D21ED21A8006C216C255
:102CE4001EC21AE53EB40413D217D21F7D037F0718
:102CF4001262534003022D7FD21B22C2178078E553
:102D04005C640F7076E53EB4010AD214D210D21C72
:102D1400D2188008C214C210C21CC218E53EB40204
:102D240013D2157D017F071262535002D211D21DB6
:102D3400D2198008C215C211C21DC219E53EB403DE
:102D440013D216D2127D027F071262535002D21E92
:102D5400D21A8008C216C212C21EC21AE53EB404B8
:102D640012D217D213D21F7D037F07126253500B66
:0B2D7400D21B22C217C213C21FC21BD9
:012D7F002231
:100FB30090001FE0540FF55CB401167D017F011210
:100FC3006253500A7F0612754D4003D20822C208AD
:100FD30022E55C6403705BE53E640170257D017F5F
:100FE30001126253500B7F0612754D4004D20880E4
:100FF30002C2087D017F021262535003D20922C24A
:101003000922E53E640260030214637D017F01123D
:1010130062535004D2088002C2087D017F0212622B
:1010230053500C7D017F071262535003D20922C231
:101033000922E55C6405705BE53E640170257D0172
:101043007F01126253500B7F0612754D4004D20884
:101053008002C2087D017F031262535003D20E2225
:10106300C20E22E53E640360030214637D017F0127
:101073001262535004D2088002C2087D017F03121A
:101083006253500C7D027F071262535003D20E222B
:10109300C20E22E55C6409705BE53E640170257D48
:1010A300017F01126253500B7F0612754D4004D22B
:1010B300088002C2087D017F041262535003D20CE0
:1010C30022C20C22E53E640460030214637D017FA7
:1010D300011262535004D2088002C2087D017F04CA
:1010E300126253500C7D037F071262535003D20CDC
:1010F30022C20C22E55C640760030211B5E53E647D
:101103000170347D017F01126253500B7F0612750B
:101113004D4004D2088002C2087D017F021262534F
:101123005004D2098002C2097D017F031262535029
:1011330003D20E22C20E22E53E640270367D017F89
:10114300011262535004D2088002C2087D017F025B
:10115300126253500D7D017F071262535004D2096E
:101163008002C2097D017F031262535003D20E2213
:10117300C20E22E53E640360030214637D017F0116
:101183001262535004D2088002C2087D017F02120A
:1011930062535004D2098002C2097D017F031262A7
:1011A30053500C7D027F071262535003D20E22C2AA
:1011B3000E22E55C640B6003021273E53E6401706A
:1011C300347D017F01126253500B7F0612754D402F
:1011D30004D2088002C2087D017F021262535004C8
:1011E300D2098002C2097D017F041262535003D2E7
:1011F3000C22C20C22E53E640270367D017F01128F
:1012030062535004D2088002C2087D017F02126239
:1012130053500D7D017F071262535004D20980029F
:10122300C2097D017F041262535003D20C22C20C07
:1012330022E53E640460030214637D017F011262B0
:10124300535004D2088002C2087D017F0212625308
:101253005004D2098002C2097D017F0412625350F7
:101263000C7D037F071262535003D20C22C20C225F
:10127300E55C640D6003021331E53E640170347D67
:10128300017F01126253500B7F0612754D4004D249
:10129300088002C2087D017F031262535004D20EFC
:1012A3008002C20E7D017F041262535003D20C22CE
:1012B300C20C22E53E640370367D017F0112625346
:1012C3005004D2088002C2087D017F03126253508A
:1012D3000D7D027F071262535004D20E8002C20EAC
:1012E3007D017F041262535003D20C22C20C22E50B
:1012F3003E640460030214637D017F011262535054
:1013030004D2088002C2087D017F03126253500495
:10131300D20E8002C20E7D017F04126253500C7DF7
:10132300037F071262535003D20C22C20C22E55CE6
:10133300640F6003021463E53E640170437D017F23
:1013430001126253500B7F0612754D4004D2088080
:1013530002C2087D017F021262535004D209800247
:10136300C2097D017F031262535004D20E8002C270
:101373000E7D017F041262535003D20C22C20C2251
:10138300E53E640270457D017F011262535004D231
:10139300088002C2087D017F02126253500D7D0155
:1013A3007F071262535004D2098002C2097D017F74
:1013B300031262535004D20E8002C20E7D017F04D9
:1013C3001262535003D20C22C20C22E53E64037016
:1013D300457D017F011262535004D2088002C20886
:1013E3007D017F021262535004D2098002C2097D3B
:1013F300017F03126253500D7D027F071262535027
:1014030004D20E8002C20E7D017F04126253500388
:10141300D20C22C20C22E53E640470447D017F019C
:101423001262535004D2088002C2087D017F021267
:1014330062535004D2098002C2097D017F03126204
:10144300535004D20E8002C20E7D017F04126253F8
:10145300500C7D037F071262535003D20C22C20C3F
:011463002266
:1078E7007F0112780A5010C209C20EC20C7F06121D
:1078F700754D500CC208227F0112780A4002C20857
:01790700225D
:107A64007F0212780A5007C209C20EC20C227F029A
:087A740012780A4002C2092247
:107A7C007F0312780A5007C209C20EC20C227F0380
:087A8C0012780A4002C20E222A
:107A94007F0412780A5007C209C20EC20C227F0466
:087AA40012780A4002C20C2214
:1069C6000500050105030507050F051F051E051C26
:1069D600051805100201040E040A03060101040B42
:1069E6000304040F020304010302040D0200020261
:1069F6000300040904040305030701000303040755
:106A0600030104060402040C05160515000006150C
:0E6A1600062A060C06380633061E0612061760
:10527000203737900640E004F519D36480948150BC
:105280000302534AD3E5196480948F400375190FC4
:1052900090063DE0FF123E6290063EE0F518E4F510
:1052A0001ED237C264C257C24A22304A60306416E6
:1052B000152EE52ED39400400302534AC2CAC2649D
:1052C000D25785182E2230570E152EE52ED3940076
:1052D0005078C264C25722AF1C151CEF700BC24A33
:1052E000E51825E0F52ED25722E51D30E00585189A
:1052F0002E8008E51875F003A4F52EAF1D7801EF98
:1053000008800103D8FDF51DD264D2CA22D5190840
:10531000C237E4F53DC25822051E7440251EF582B1
:10532000E43406F583E025E024C6F582E43469F52B
:1053300083E493540FF51C740193F51D700AD25742
:0A534000E51825E025E0F52ED24A1D
:01534A002240
:105F790020371A90063DE0FF123E6290063EE0F59A
:105F89001AE4F51ED237C264C257C24A22304A59AE
:105F9900306413152EE52ED39400506BC2CAC26427
:105FA900D257851A2E2230570E152EE52ED394007E
:105FB9005055C264C25722AF1C151CEF7007C24A64
:105FC900C237F53D22E51D30E005851A2E8008E52A
:105FD9001A75F003A4F52EAF1D7801EF08800103AF
:105FE900D8FDF51DD264D2CA22E53F25E024C6F5C5
:105FF90082E43469F583E493FA740193FBEA540F5C
:07600900F51CEBF51DD24A66
:01601000226D
:107B2900C3EF648094A15008EF25E025E0F52E22EB
:047B3900E4F52E221F
:10747E00BF010790063E7418F022BF020790063E29
:10748E007412F022BF030590063E8014BF040790CD
:10749E00063E740BF02290063EBF05047409F022DE
:0474AE00740CF02248
:103E6200EF14B420004003023FB5903E7A75F00390
:103E7200A4C58325F0C58373023EDA023EE1023E09
:103E8200E8023EEF023EF6023EFD023F04023F0B15
:103E9200023F12023F19023F20023F27023F2E0239
:103EA2003F35023F3C023F43023F4A023F51023F3D
:103EB20058023F5F023F66023F6D023F74023F7B42
:103EC200023F82023F89023F90023F97023F9902DE
:103ED2003FA0023FA7023FAE75CB8E75CAC62275C0
:103EE200CB9575CA772275CB9B75CA692275CBA013
:103EF20075CABA2275CBA675CA332275CBAB75CA01
:103F0200632275CBB075CA022275CBB475CAA322DF
:103F120075CBB875CAFA2275CBBC75CAD82275CBD7
:103F2200C075CAA82275CBC475CA362275CBC775AF
:103F3200CA862275CBCA75CABC2275CBCD75CAB4E6
:103F42002275CBD075CA762275CBD375CA3022754D
:103F5200CBD575CAB22275CBD875CA132275CBDA06
:103F620075CA522275CBDC75CA7D2275CBDD75CA46
:103F72006E2275CBE075CA542275CBE275CA1B223C
:103F820075CBE375CAC32275CBE575CA5E2275CBC4
:103F9200E675CADA22801C75CBE875CA902275CB09
:103FA200EA75CAD92275CBEC75CA092275CBED75B3
:0A3FB200CA292275CBE875CA412226
:1071D200EFC39400403FEF9408503AE4FEEF75F09D
:1071E20008A42430F582E43400F583E5822EF5828A
:1071F200E43583F583E0FCED75F008A424E8F5821C
:10720200E4341AF583E5822EF582E43583F583ECC6
:05721200F00EBE08C8EB
:017217002254
:1060A7008F5BE55B6405701D200A0DD20A7FF47EC5
:1060B70001127A15C20A8074C20A7FF47E01127A2D
:1060C70015D20A8067E55B6406701D200B0DD20BA5
:1060D7007FF47E01127A15C20B800BC20B7FF47E10
:1060E70001127A15D20B8044E55B6407701D200FFF
:1060F7000DD20F7FF47E01127A15C20F800BC20FEB
:106107007FF47E01127A15D20F8021E55B64087057
:1061170022200D0DD20D7FF47E01127A15C20D805B
:106127000BC20D7FF47E01127A15D20D7FF47E012A
:04613700127A1522A1
:104DA900A233B330B401B350357D017F0812625389
:104DB9005027A233B35010A2B4B3500B900652E05F
:104DC900FF7C077D30800F30330F30B40C900653D1
:104DD900E0FF7C077D501272E3A2B4B39233A23490
:104DE900B330B501B350357D027F081262535027A5
:104DF900A234B35010A2B5B3500B900654E0FF7C17
:104E0900077D70800F30340F30B50C900655E0FFE8
:104E19007C077D901272E3A2B5B39234A235B33008
:104E2900B701B350357D037F081262535027A2356D
:104E3900B35010A2B7B3500B900656E0FF7C077D24
:104E4900B0800F30350F30B70C900657E0FF7C0764
:104E59007DD01272E3A2B7B39235A236B330B60150
:104E6900B350357D047F081262535027A236B350E0
:104E790010A2B6B3500B900658E0FF7C077DF08076
:104E89000F30360F30B60C900659E0FF7C087D10C4
:094E99001272E3A2B6B3923622B4
:10766A00900027E0FF30E404D20A8002C20AEF3019
:10767A00E504D20B8002C20BEF30E604D20F80027F
:0B768A00C20FEF30E703D20D22C20D4B
:0176950022D2
:1074130090063CE0FF602E20370F6029123E62D2B7
:10742300CAD237D264752E1422E52ED394004003BA
:10743300152E22206408D2CA752E14D26422C2CA21
:06744300752E7DC26422DB
:107449002037127F1C123E62D2CAD237D264752EFF
:1074590064751B3C22E52ED394004003152E22AF00
:107469001B151BD3EF648094804004752E6422C2DF
:0474790037E4F53DC2
:01747D0022EC
:104EA20020371C754006E53E75F008A424E8F5821B
:104EB200E4341AF583E06003D23722E4F53D22E5BB
:104EC2002ED394004003152E22C2CA1540E5401489
:104ED2007003024F5D14606F14604014602E146002
:104EE20003024F91E53E75F008A424E8F582E4340C
:104EF2001AF583E0FF7003F53D22123E62E53E752E
:104F0200F008A424E9F582E4341A8079E53E75F0CC
:104F120008A424EAF582E4341A80397408441B7028
:104F220003F53D22E53E75F008A424EBF582E43456
:104F32001AF583E0FF123E62E53E75F008A424EC08
:104F4200F582E4341A803EE53E75F008A424EDF5BE
:104F520082E4341AF583E0FF027B297420441B703B
:104F620003F53D22E53E75F008A424EEF582E43413
:104F72001AF583E0FF123E62E53E75F008A424EFC5
:104F8200F582E4341AF583E0FF127B29D2CA22E4C7
:074F9200F53DC2CAC237223F
:1074B200E53D14601C14601C14601C14601F1460F1
:1074C2001F2405701EC2CAC237C264C257E4F54007
:1074D20022024EA2027413125270D258220274492E
:0474E200125F79229A
:10761000E52365437004E5226542601F85224285AB
:107620002343C2A4D2A5C2A6C2A700AF23127AC226
:0D763000E522FF127AC200D2A7D322C322A6
:1079DD00E52465446014852444D2A4D2A5C2A6C270
:0C79ED00A7AF24127AC2D2A7D322C32273
:1079F900E521653C601485213CD2A4C2A5C2A6C27A
:0C7A0900A7AF21127AC2D2A7D322C32259
:10410800E4F54CF54D754E1E754FFF854D82854C77
:1041180083E0F5506350FFE550F0E065506003120E
:104128007BB96350FF854D82854C83E550F0E0658F
:10413800506003127BB9054DE54D7002054CE54F03
:10414800154F7002154ED3E54F9400E54E9400507C
:10415800BAE4F54CF54DF54EF54FE54D254FF58292
:10416800E54C354EF583E4F0054FE54F7002054EFA
:10417800B4FFE7E54EB41EE275985A758921758833
:1041880045758845758DE775878075C90275331B38
:1041980075341075351B75366075371B7538B075F5
:1041A800391C753A0075B701D2A9D2A8D2AA9006CF
:1041B80000E0FFA3E0901CE0CFF0A3EFF090060230
:1041C800E0FFA3E0901CE2CFF0A3EFF0900604E03C
:1041D800FFA3E0901CE4CFF0A3EFF0900606E0FF09
:1041E800A3E0901CE6CFF0A3EFF0901CFA7417F050
:1041F800A37499F0901CFC7417F0A37499F0901CA8
:10420800FE7417F0A37499F0901D007417F0A3744E
:0942180099F0D291D2AF1277188F
:01422100227A
:027BB90080FE4C
:10754D00C2AFC284D285BF060AC286E580A2E1928F
:10755D006B8018BF070AC286E580A2E2926B800B92
:10756D00BF0808C286E580A2E3926BD286D2AFA295
:01757D006BA2
:01757E0022EA
:10625300BF0107900020E0FE8048BF0207900021A5
:10626300E0FE803EBF0307900022E0FE8034BF04BF
:1062730007900023E0FE802ABF0507900024E0FE7C
:106283008020BF0607900025E0FE8016BF07079019
:106293000026E0FE800CBF0807900027E0FE800286
:1062A300E4FEBD0103EE1322BD0204EEA2E122BD12
:1062B3000304EEA2E222BD0404EEA2E322BD050420
:1062C300EEA2E422BD0604EEA2E522BD0704EEA27F
:0762D300E622BD0802EE33D4
:0162DA0022A1
:024F99008F4D3A
:104F9B009000B0E0F54EE54D64017037E54E24020C
:104FAB00FFE433FE7868E66F7001EE600302508E0B
:104FBB007410254EF582E4341BAF82F5508F51D21D
:104FCB006B7F01125A491279A312385DC26B7F01B4
:104FDB0002508BE54D64027037E54E2402FFE4333B
:104FEB00FE7869E66F7001EE600302508E746025E7
:104FFB004EF582E4341BAF82F5508F51D26B7F029A
:10500B00125A491279A312385DC26B7F0202508B80
:10501B00E54D64037033E54E2402FFE433FE786AFA
:10502B00E66F7001EE705C74B0254EF582E4341BB4
:10503B00AF82F5508F51D26B7F03125A491279A36D
:10504B0012385DC26B7F038037E54D64047034E525
:10505B004E2402FFE433FE786BE66F7001EE702393
:10506B007400254EF582E4341CAF82F5508F51D27B
:10507B006B7F04125A491279A312385DC26B7F04FD
:03508B00125A496D
:01508E0022FF
:04385D008F4FE4FDA8
:023861008D5781
:1038630075F020EFA42460F582E5F03403AF82F510
:103873005A8F5BF583E0F558D3940050030239EB7C
:10388300E558941040030239EBE557704C7FF47E02
:1038930001127A15E55825E0F558755901E55824C4
:1038A30001FFE433FEC3E5599FEE6480F87480980A
:1038B30040030239EBE55B2559F582E4355AF5837C
:1038C300E0FFE55B2559F582E4355AF583A3E0FD76
:1038D3001276EE0559055980C4E5576401707AC222
:1038E3002B7FF47E01127A15E55825E0F5587559BA
:1038F30001E5582401FFE433FEC3E5599FEE6480DC
:10390300F874809840030239EBE55B2559F582E4AE
:10391300355AF583E0FFE55B2559F582E4355AF521
:1039230083A3E0FD1276EE90001FE0FF30E0063047
:103933004903C22022EF30E106304D03C22122EFBA
:1039430030E206305103C22222EF30E30630540343
:10395300C22322055905598098E557640260030282
:1039630039EBC22BC22CC22DC22E7FF47E01127AF8
:1039730015E55825E0F558755901E5582401FFE48C
:1039830033FEC3E5599FEE6480F87480985059E57F
:103993005B2559F582E4355AF583E0FFE55B25594C
:1039A300F582E4355AF583A3E0FD1276EE90001F0D
:1039B300E030E005303902802290001FE030E1055D
:1039C300303A02801690001FE030E205303B02805F
:1039D3000A90001FE030E30A303C07C220C26902AC
:0839E300721805590559809284
:0139EB0022B9
:02455F008F4D7E
:10456100C2679000A8E0FFE54DB401167868E6FE49
:10457100D39F400EEE9FF55074102FF582E4341B4B
:10458100804FE54DB402167869E6FED39F400EEEEA
:104591009FF55074602FF582E4341B8034E54DB4EF
:1045A1000316786AE6FED39F400EEE9FF55074B075
:1045B1002FF582E4341B8019E54DB4041C786BE6B9
:1045C100FED39F4014EE9FF55074002FF582E43422
:1045D1001CAF82F5518F52D26720670302466FD21A
:1045E1006BAF4D125A497FF47E01127A157D207FFF
:1045F100051276EE7D1A7F081276EE7FC87E0012D4
:104601007A15E4F54EE54EC39550505B0552E552DF
:10461100AE517002055114F5828E83E0F54F60367C
:1046210024F5601414601714601A14601D146020BE
:1046310024057028E4FD80277D5F7F0780227D5E51
:104641007F06801C7D0A7F0280167D327F028010EA
:104651007D467F02800A7D0A7F038004AD4FE4FF1F
:0E4661001276EE054E809EC26BAF4D125A4986
:01466F002228
:10776B0030290F900671E0FF7C0B7D101272E3B293
:10777B002922202912900670E0FF7C0A7DF01272FC
:08778B00E3B229E4786CF62258
:106011007D3F7F091276EE7D507F081276EE90006B
:106021000EE493FDE4FF1276EE7D5B7F061276EEC1
:1060310090000FE493FDE4FF1276EE900010E493DC
:10604100FDE4FF1276EE900011E49324BFB4080042
:10605100505390606175F003A4C58325F0C5837327
:1060610002607902607D02608102608702608D02B8
:10607100609302609902609F7D0A80067D328002F2
:106081007D467F02801C7D0A7F0380167D287F0369
:1060910080107D467F03800A7D0A7F0480047D286D
:0660A1007F041276EE22DE
:1077E3008F53D26B125A497D4B7F021276EE7D0482
:1077F300E4FF1276EE7D387F041276EE126011C23A
:077803006BAF53125A49223A
:0B79A300855182855083E0FFA3E0FDCA
:1079AE00BF0A02E4FFBD0A02E4FDEF75F00AA42D42
:0279BE00FF22A6
:10534B00C267D208D2207FF47E01127A157D2E7FA0
:10535B00031276EE7D607F021276EEC208C2201237
:10536B0033467F0812754D40030254173049F01233
:10537B0033462049FA7868E6640770427E007F70F6
:10538B0075331B7534108F828E837407F07D01E5A6
:10539B00342DF582E43533F583E58224FFF582E580
:1053AB008334FFF583E0F9EF2DF582E43EF583E9D5
:1053BB00F00DBD08DAD2677F647E00127A157F0884
:1053CB0012754D504720670302534DD208D2207FF0
:1053DB00F47E01127A157D607F021276EE7D327FAC
:1053EB00061276EE7D1E7F051276EEC208C2207C79
:1053FB00007D707B087F787E001267C97F0812756D
:10540B004D50097F327E00127A1580F0126CEC7FC2
:06541B00647E00127A1508
:015421002268
:10774200E4F53DC258C258F532302F05C22FC23F70
:1077520022303005C230C24122303105C231C2432B
:0977620022303204C232C2452279
:104222007580FFC286E580540FFFC285E580C454C5
:10423200F04FF520D2867D027F0112625340107D3D
:10424200037F011262534007300004D23980287D77
:10425200027F01126253500A300007300104D23942
:1042620080157D037F01126253500A200003300142
:1042720004D2398002C2397D027F02126253401099
:104282007D037F021262534007300204D23A802833
:104292007D027F02126253500A300207300304D2B9
:1042A2003A80157D037F02126253500A20020330C6
:1042B2000304D23A8002C23A7D027F031262534063
:1042C200107D037F031262534007300404D23B8007
:1042D200287D027F03126253500A3004073005041E
:1042E200D23B80157D037F03126253500A200403E0
:1042F200300504D23B8002C23B7D027F041262532E
:10430200400F7D037F041262534006300603D23C05
:10431200227D027F041262535009300606300703E1
:10432200D23C227D037F04126253500920060330DF
:074332000703D23C22C23C4C
:014339002261
:10334600202B6EC25A20391C205019901CFAE070AE
:1033560002A3E0700B7D067F011262535002D24732
:10336600C249804D30392130501E901CE0E0700279
:10337600A3E0700B7D087F011262535002D23D30EC
:103386006502D25BD2498029303908205005126C7B
:10339600EC801E20391B305018D25AC249C250C286
:1033A60014C210C21CC2181278E77868E66002D20E
:1033B6005B202C71203A1C205319901CFCE07002F3
:1033C600A3E0700B7D067F021262535002D24BC2FD
:1033D6004D8052303A28305325901CE2E07002A30B
:1033E600E070127D087F0212625350097F02127844
:1033F6000A5002D23E306602D25BD24D8027303A66
:1034060008205305126D40801C203A19305316C20D
:103416004DC253C215C211C21DC219127A6478690F
:10342600E66002D25C202D71203B1C205519901CB1
:10343600FEE07002A3E0700B7D067F03126253501C
:1034460002D24EC2518052303B28305525901CE4A2
:10345600E07002A3E070127D087F031262535009E8
:103466007F0312780A5002D240302802D25BD25132
:103476008027303B08205505126D94801C203B198F
:10348600305516C251C255C216C212C21EC21A12F7
:103496007A7C786AE66002D25D202E6D203C1B2085
:1034A6005618901D00E07002A3E0700B7D067F04A5
:1034B6001262535002D252C25422303C2730562454
:1034C600901CE6E07002A3E070127D087F04126291
:1034D6005350097F0412780A5002D242302A02D28F
:1034E6005BD25422303C06205603026DE8203C197C
:1034F600305616C254C256C217C213C21FC21B127E
:0A3506007A94786BE66002D260222E
:047BB20012508F22BC
:10508F0090001FE0540FFFBF010B304906203D0376
:10509F00025156C322EF64037014304906203D03BA
:1050AF00025156304D06203E03025161C322EF6478
:1050BF00057014304906203D030251563051062029
:1050CF00400302516CC322EF64097013304905206D
:1050DF003D028073305406204203025177C322EF02
:1050EF006407701A304905203D02805B304D052062
:1050FF003E02805E3051052040028061C322EF6482
:10510F000B701A304905203D02803C304D05203E82
:10511F0002803F305405204202804DC322EF640DC0
:10512F00701A304905203D02801D30510520400284
:10513F00802B305405204202802EC322EF640F7063
:10514F002E304908203D05753E01D322304D0820F1
:10515F003E05753E02D322305108204005753E03AF
:10516F00D322305408204205753E04D322C322C3F4
:01517F00220D
:10780A00BF010690001FE01322BF020790001FE08D
:10781A00A2E122BF030790001FE0A2E222BF0406F2
:07782A0090001FE0A2E32221
:106CEC007868E6602275331B753410E4FFE5342FA9
:106CFC00F582E43533F583E4F00FBF50F075331BA8
:106D0C00753410E47868F6900600E0FFA3E0901C60
:106D1C00E0CFF0A3EFF0900608E0FFA3E0901CFAA0
:106D2C00CFF0A3EFF0C246C247C25FC23DC265C2FC
:036D3C003FD250F3
:016D3F002231
:106D40007869E6602275351B753660E4FFE5362FFD
:106D5000F582E43535F583E4F00FBF50F075351B4F
:106D6000753660E47869F6900602E0FFA3E0901CB7
:106D7000E2CFF0A3EFF090060AE0FFA3E0901CFC46
:106D8000CFF0A3EFF0C248C24BC261C23EC266C29E
:036D900041D2539A
:016D930022DD
:106D9400786AE6602275371B7538B0E4FFE5382F52
:106DA400F582E43537F583E4F00FBF50F075371BF7
:106DB4007538B0E4786AF6900604E0FFA3E0901C0E
:106DC400E4CFF0A3EFF090060CE0FFA3E0901CFEEC
:106DD400CFF0A3EFF0C24CC24EC262C240C228C27E
:036DE40043D25542
:016DE7002289
:106DE800786BE6602275391C753A00E4FFE53A2FA6
:106DF800F582E43539F583E4F00FBF50F075391C9E
:106E0800753A00E4786BF6900606E0FFA3E0901C64
:106E1800E6CFF0A3EFF090060EE0FFA3E0901D0090
:106E2800CFF0A3EFF0C24FC252C263C242C22AC21D
:036E380045D256EA
:016E3B002234
:10599400C208C209C20EC20C1279F9C267D25EE40F
:1059A400F53D7FE87E03127A15C298C2AF75567F23
:1059B400755596755498755300785374FF1259763B
:1059C400E4FBFAF9F8C3125963504430983E1200CC
:1059D40006127B74EF14601824F0602624C1600B57
:1059E40024F670287F06127BA28021127142801C4B
:1059F4007F06127BA21274E612766A126FD0D26707
:105A0400800A7F06127BA2126758D2673067AAE425
:105A1400786CF6D26B7F01125A497F01126BEC7DD0
:105A2400467F021276EE7D1E7F071276EE7D147F8E
:105A3400081276EE7D327F031276EEC26B7F01127E
:045A44005A49C25E9B
:015A4800223B
:10675800756701756500756620E4F5577F02127B41
:10676800A2E5672402F559AF67127BA2E4F558E564
:10677800662558F582E43565F583E0FF127BA2E5CE
:10678800662558F582E43565F583E02559F5590500
:1067980058E558C3948040D7AF59127BA27F0312A3
:1067A8007BA2127BAAEF64156016056774802566C4
:1067B800F566E43565F5650557E557C39435409C9E
:0167C80022AE
:1074E600756701756500756620E4F55712763D509F
:1074F600077F06127BA280057F15027BA2056774B3
:10750600802566F566E43565F5650557E557C39448
:037516003540D924
:01751900224F
:10763D00E4F558127BAA74502558F582E4341CF5F4
:10764D0083EFF00558E558C3948440E7127AD8903B
:0C765D001CD2E0B50705127908D322C347
:0176690022FE
:10790800E4FF74522FF582E4341CF583E0FEE5664B
:0F7918002FF582E43565F583EEF0000FBF80E3B5
:01792700223D
:107AD800E4FFFE74502EF582E4341CF583E02FFF9A
:047AE8000EBE82EF5D
:017AEC002277
:10714200E4F557F55D755CE0755B93755A04F55986
:10715200785974FF125976E4FBFAF9F8C3125963AD
:1071620050253098EB1200068F58E55864046017DA
:10717200AF5D055D74502FF582E4341CF583E5584C
:07718200F02557F55780C905
:0171890022E3
:04000600AF99C29854
:01000A0022D3
:087BA2003099FDC2998F992270
:077BAA003098FDAF99C2986D
:017BB10022B1
:105BB100070102030405060707070605040302019E
:105BC10003010A0A03020A0A03030A0A03040A0A6E
:105BD100030307050303020503070A0A04024B0036
:105BE100040438072E03024B0004043802055F0049
:105BF1000302055F000402055F000502055F000660
:105C010002055F000702055F000802055F00090247
:105C1100055F000A02055F000B02055F000C02052B
:105C21005F000D02055F000E02055F000F02055FB8
:105C3100001002055F001102055F001204072E0823
:105C4100260640033204072E082606400253080C9C
:075C51000A1D040000241BE2
:10001600C2AF9000207491F09000217481F090009E
:1000260022F0900023F09000247403F090002574D1
:10003600BFF09000267408F0900027740FF090002F
:10004600307409F0A37403F0E4A3F0A37410F0A3D2
:100056007403F0E4A3F0A37415F0A37403F0A3747F
:1000660015F0A37403F0E4A3F0A37410F0A37403D3
:10007600F0E4A3F0A37409F0A37403F0A37415F0DD
:10008600A37403F0A314F0A3741AF0A37403F0E4AA
:10009600A3F0A3F0A3F0A3741AF0A37403F0A314BF
:1000A600F0A37415F0A37403F0E4A3F0A3F0A3F097
:1000B6007E5B7FC17C007D807B041272A27E5B7FAB
:1000C600C57C007D887B041272A27E5B7FC97C00A2
:1000D6007D907B041272A27E5B7FCD7C007D987B37
:1000E600041272A27E5B7FD57C007DA07B04127217
:1000F600A27E5B7FD17C007DA87B041272A27E5B10
:100106007FD97C007DB07B041272A27E5B7FB17CBE
:10011600007D707B081272A27E5B7FB97C007D78C1
:100126007B081272A27E5B7FDD7C037D807B0912D9
:1001360072A27E5B7FE67C037DA07B071272A27EA5
:100146005B7FED7C037DC07B051272A27E5B7FF236
:100156007C037DE07B051272A27E5B7FF77C047DCB
:10016600007B051272A27E5B7FFC7C047D207B05F2
:100176001272A27E5C7F017C047D407B051272A216
:100186007E5C7F067C047D607B051272A27E5C7FAE
:100196000B7C047D807B051272A27E5C7F107C0442
:1001A6007DA07B051272A27E5C7F157C047DC07BE0
:1001B600051272A27E5C7F1A7C047DE07B051272BA
:1001C600A27E5C7F1F7C057D007B051272A27E5C91
:1001D6007F247C057D207B051272A27E5C7F297CB4
:1001E600057D407B051272A27E5C7F2E7C057D60BC
:1001F6007B051272A27E5C7F337C057D807B0512B7
:1002060072A27E5C7F387C057DA07B051272A27E81
:100216005C7F3D7C057DC07B091272A27E5C7F46B9
:100226007C057DE07B091272A2900600E4F0A374BF
:10023600B4F0900602E4F0A374B4F0900604E4F07F
:10024600A374B4F0900606E4F0A374B4F090061814
:100256007401F0A374E0F090061AE4F0A37478F049
:1002660090061EE4F0A3743CF09006087402F0A316
:100276007458F090060A7402F0A37458F090060CB5
:100286007402F0A37458F090060E7402F0A374582A
:10029600F09006107401F0A3742CF090061274020C
:1002A600F0A37458F09006147403F0A37484F090CD
:1002B60006167404F0A374B0F07407900620F0A339
:1002C600F0900622F0A3F090061C7402F0A3745876
:1002D600F0900630740AF09006317428F0900633D8
:1002E600740AF0900634F09006327405F07E5C7F56
:1002F6004F7C067D407B091272A290063D7417F072
:1003060090063E740CF090063C7419F0E490063F9B
:10031600F090063B740CF09006527401F090073092
:100326007469F0A37411F09006537401F0900750AD
:100336007469F0A37410F09006547401F09007707D
:100346007469F0A37421F09006557401F09007903B
:100356007469F0A37420F09006567401F09007B00B
:100366007469F0A37431F09006577401F09007D0C9
:100376007469F0A37430F09006587401F09007F099
:100386007469F0A37441F09006597401F090081056
:100396007469F0A37440F090065A7401F090083026
:1003A6007462F0A37411F0A37432F0A37401F0A385
:1003B6007450F0A37410F090065B7401F09008502E
:1003C6007461F0A37420F0A37462F0A37411F0A317
:1003D6007432F0A37402F0A37450F0A37410F0907A
:1003E600065C7401F09008707451F0A37411F0A3C8
:1003F6007433F0A3E4F0A37451F0A37410F09006E4
:100406005D7401F09008907462F0A37411F0A37407
:1004160030F0A37402F0A37462F0A37410F0900697
:100426005E7401F09008B07451F0A37411F0A374D7
:1004360041F0A37410F0A37451F0A37410F0900669
:100446005F7401F09008D07451F0A37411F0A37496
:1004560034F0A37414F0A37451F0A37410F0900652
:10046600607401F09008F07451F0A37411F0A37455
:1004760034F0A37418F0A37451F0A37410F090062E
:10048600617401F09009107451F0A37411F0A37413
:1004960034F0A37428F0A37451F0A37410F09006FE
:1004A600627401F09009307462F0A37411F0A374C1
:1004B60030F0A37403F0A37462F0A37410F09006F6
:1004C600637401F09009507462F0A37411F0A37480
:1004D60030F0A37404F0A37462F0A37410F09006D5
:1004E600647401F09009707462F0A37411F0A3743F
:1004F60060F0A37401F0A37495F0A3743DF0A374A7
:1005060090F0A37401F0A37498F0A37426F0A3747A
:1005160096F0A37440F0A37462F0A37410F0A37471
:1005260061F0A37470F09006657401F09009907400
:1005360062F0A37411F0A37460F0A37401F0A374C5
:1005460095F0A3743DF0A37490F0A37401F0A37426
:1005560096F0A37438F0A37462F0A37410F09006BA
:10056600667401F09009B07462F0A37411F0A3747C
:1005760060F0A37401F0A37495F0A3743DF0A37426
:1005860090F0A37402F0A37498F0A37426F0A374F9
:1005960096F0A37440F0A37462F0A37410F0A374F1
:1005A60061F0A37470F09006677401F09009D0743E
:1005B60062F0A37411F0A37460F0A37401F0A37445
:1005C60095F0A3743DF0A37490F0A37402F0A374A5
:1005D60096F0A37438F0A37462F0A37410F090063A
:1005E600687401F09009F07462F0A37411F0A374BA
:1005F60060F0A37401F0A37495F0A3743DF0A374A6
:1006060090F0A37403F0A37498F0A37426F0A37477
:1006160096F0A37440F0A37462F0A37410F0A37470
:1006260061F0A37470F09006697401F0900A10747A
:1006360062F0A37411F0A37460F0A37401F0A374C4
:1006460095F0A3743DF0A37490F0A37403F0A37423
:1006560096F0A37438F0A37462F0A37410F09006B9
:100666006A7401F0900A307462F0A37411F0A374F6
:1006760060F0A37401F0A37495F0A3743DF0A37425
:1006860090F0A37404F0A37498F0A37426F0A374F6
:1006960096F0A37440F0A37462F0A37410F0A374F0
:1006A60061F0A37470F090066B7401F0900A5074B8
:1006B60062F0A37411F0A37460F0A37401F0A37444
:1006C60095F0A3743DF0A37490F0A37404F0A374A2
:1006D60096F0A37438F0A37462F0A37410F0900639
:1006E6006C7401F0900A707462F0A37411F0A37434
:1006F60060F0A37401F0A37430F0A37405F0A37442
:1007060062F0A37410F090066D7401F0900A907474
:1007160062F0A37421F0A37460F0A37401F0A374D3
:1007260030F0A37406F0A37462F0A37420F0900670
:100736006E7401F0900AB07462F0A37431F0A37481
:1007460060F0A37401F0A37430F0A37407F0A374EF
:1007560062F0A37430F090066F7401F0900AD074C2
:1007660062F0A37441F0A37460F0A37401F0A37463
:1007760030F0A37408F0A37462F0A37440F09006FE
:10078600707401F0900AF07464F0A37411F0A3740D
:1007960096F0A37432F0A37495F0A3741EF0A374BC
:1007A60098F0A3744BF0A37464F0A37410F0900651
:1007B600717401F0900B107464F0A37411F0A374BB
:1007C60096F0A37432F0A37495F0A3741EF0A3748C
:1007D60093F0A37418F0A37464F0A37410F0900659
:1007E600737401F0900B507462F0A37411F0A3744B
:1007F60060F0A37401F0A37495F0A3743DF0A374A4
:1008060090F0A37402F0A37497F0A37426F0A37477
:1008160093F0A37418F0A37462F0A37410F0A37499
:1008260070F0A37410F09006747401F0900B70745D
:1008360062F0A37411F0A37460F0A37401F0A374C2
:1008460095F0A3743DF0A37490F0A37403F0A37421
:1008560097F0A37426F0A37493F0A37418F0A3740E
:1008660062F0A37410F0A37470F0A37420F09006E5
:10087600757401F0900B907462F0A37411F0A37478
:1008860060F0A37401F0A37495F0A3743DF0A37413
:1008960090F0A37404F0A37497F0A37426F0A374E5
:1008A60093F0A37418F0A37462F0A37410F0A37409
:1008B60070F0A37430F09006817401F0900D1074FE
:1008C60062F0A37411F0A37460F0A37401F0A37432
:1008D60092F0A3744BF0A37490F0A37404F0A37485
:1008E60094F0A37438F07499A3F0A3F0A37460F0A5
:1008F600A37401F0A37462F0A37410F01222F8122C
:100906006FD0D26B7F01125A497D2F7F071276EE88
:100916007D0C7F031276EE7D327F061276EE7D1E0B
:100926007F051276EE90001F7401F0FD7F1F7E009A
:0B093600127323C26B7F01125A49228A
:1022F8009001007402F0A3740DF0A37402F090062C
:10230800A014F09010F07464F0A37411F0A3749703
:10231800F0A3742EF0A37495F0A3743DF0A3749009
:10232800F0A37402F0A37496F0A37438F0A3746455
:10233800F0A37410F0A37470F0A37411F090010866
:102348007402F0A3740EF0A37402F09006A114F0C6
:102358009011107461F0A37410F0A37464F0A37466
:1023680011F0A37497F0A3742EF0A37495F0A374DE
:102378003DF0A37490F0A37402F0A37496F0A374D4
:1023880036F0A37464F0A37410F0A37470F0A3740F
:1023980010F09001107402F0A3740DF0A37403F010
:1023A8009006A27401F09011307464F0A37411F0D7
:1023B800A37497F0A3742EF0A37495F0A3743DF062
:1023C800A37490F0A37403F0A37496F0A37438F088
:1023D800A37464F0A37410F0A37470F0A37421F0D4
:1023E8009001187402F0A3740EF0A37403F0900621
:1023F800A37401F09011507461F0A37410F0A374E9
:1024080064F0A37411F0A37497F0A3742EF0A3746E
:1024180095F0A3743DF0A37490F0A37403F0A37433
:1024280096F0A37436F0A37464F0A37410F0A37448
:1024380070F0A37420F09001207402F0A3740DF0E2
:10244800A37404F09006A47401F09011707464F001
:10245800A37411F0A37497F0A3742EF0A37495F0ED
:10246800A3743DF0A37490F0A37404F0A37496F0E1
:10247800A37438F0A37464F0A37410F0A37470F01C
:10248800A37431F09001287402F0A3740EF0A374C1
:1024980004F09006A57401F09011907461F0A37493
:1024A80010F0A37464F0A37411F0A37497F0A374EC
:1024B8002EF0A37495F0A3743DF0A37490F0A37468
:1024C80004F0A37496F0A37436F0A37464F0A374B4
:1024D80010F0A37470F0A37430F09001307403F01E
:1024E800A3740DF0A37402F0A304F09006A674017F
:1024F800F09011B07464F0A37411F0A37497F0A372
:10250800742EF0A37495F0A3743DF0A37490F0A317
:102518007402F0A37490F0A37403F0A37496F0A36C
:102528007438F0A37464F0A37410F0A37470F0A36B
:102538007441F09001387403F0A3740EF0A3740290
:10254800F0A304F09006A77401F09011D07461F024
:10255800A37410F0A37464F0A37411F0A37497F03B
:10256800A3742EF0A37495F0A3743DF0A37490F0B7
:10257800A37402F0A37490F0A37403F0A37496F00C
:10258800A37436F0A37464F0A37410F0A37470F00D
:10259800A37440F09001407404F0A3740DF0A37488
:1025A80002F0A304F0A304F09006A87401F09011BF
:1025B800F07464F0A37411F0A37497F0A3742EF070
:1025C800A37495F0A3743DF0A37490F0A37402F083
:1025D800A37490F0A37403F0A37490F0A37404F0B0
:1025E800A37496F0A37438F0A37464F0A37410F085
:1025F800A37470F0A37441F0A37470F0A37451F045
:102608009001487404F0A3740EF0A37402F0A304BC
:10261800F0A304F09006A97401F09012107461F010
:10262800A37410F0A37464F0A37411F0A37497F06A
:10263800A3742EF0A37495F0A3743DF0A37490F0E6
:10264800A37402F0A37490F0A37403F0A37490F041
:10265800A37404F0A37496F0A37436F0A37464F022
:10266800A37410F0A37470F0A37440F0A37470F016
:05267800A37450F022E4
:0A72A2008E4C8F4D8C4E8D4F8B509B
:1072AC00E4F9C3E5506480F8E96480985028E9FF5C
:1072BC003395E0FEE54D2FF582E54C3EF583E493E6
:1072CC00FFE9FD3395E0FCE54F2DF582E54E3CF5ED
:0672DC0083EFF00980CCF5
:0172E2002289
:107A4A00D291C2A4C2A5C2A6C2A7007F05127AC259
:097A5A0000127AAC00D2A7D2910F
:017A63002200
:10796700127A4AEF20E0F9D291C2A4C2A5C2A6C2F8
:0E797700A7007F06127AC20000D2A7D291228A
:10798500127A4AEF20E0F9D291C2A4C2A5C2A6C2DA
:0E799500A7007F04127AC20000D2A7D291226E
:046E3C008E528F5390
:106E4000AE04AF058E568F57D291C2A4C2A5C2A67A
:106E5000C2A7007F03127AC2E552FF127AC2AF5373
:106E6000127AC2E4F554F555127AACE5572555F57A
:106E700082E5563554F583EFF00555E5557002056A
:0E6E800054C39420E554940040DED2A7D29172
:016E8E0022E1
:086907008E5D8F5E8C5F8D60D8
:10690F00127A4AEF20E0F9127967855D63855E643C
:10691F00D291C2A4C2A5C2A6C2A7007F02127AC298
:10692F00E55FFF127AC2AF60127AC2E4F561F562D9
:10693F00E5642562F582E5633561F583E0FF127A40
:10694F00C20562E56270020561C39420E56194009F
:07695F0040DE00D2A7D29137
:01696600220E
:0A67C9008E4C8F4D8C4E8D4F8B507F
:1067D300C2AF127967127A4AEF20E0F9854E5285EB
:1067E3004F53D291C2A4C2A5C2A6C2A7007F021270
:1067F3007AC2E54CFF127AC2AF4D127AC2E4F55168
:10680300AF50EF3395E0FEC3E5519FEE6480F8741B
:1068130080985014E5532551F582E43552F583E011
:10682300FF127AC2055180D800D2A7D2911279857E
:02683300D2AFE2
:016835002240
:107323008E5B8F5C8D5DC2AF127967127A4AEF2054
:10733300E0F9D291C2A4C2A5C2A6C2A7007F0212DD
:107343007AC2E55BFF127AC2AF5C127AC2AF5D12FA
:0E7353007AC20000D2A7D291127985D2AF2261
:047831008E4C8F4D9D
:10783500D291C2A4C2A5C2A6C2A77F03127AC2E58D
:107845004CFF127AC2AF4D127AC2127AACD2A7D2CD
:0178550091A1
:01785600220F
:10718A00C2AF754E00754F20755000755120E4F559
:10719A004CF54DAD4FAC4EAF51AE50126E3C742013
:1071AA00254FF54FE4354EF54E74202551F551E43F
:1071BA003550F550054DE54D7002054CC394D6E5A2
:0771CA004C940040CED2AF4F
:0171D100229B
:106FD000C2AF755B00755C20755900755A20E4F5E9
:106FE00057F558AD5AAC59AF5CAE5B1269077420C7
:106FF000255AF55AE43559F5597420255CF55CE4B9
:10700000355BF55B0558E55870020557C394D6E526
:0A70100057940040CE127985D2AFEC
:01701A002253
:046EE1008C4D8D4EF9
:106EE500EF6048D22BD22CD22DD22EE4F54F854E11
:106EF50082854D83E0FEA3E04E6028AF4FEF3395CA
:106F0500E0FEEF25E0FFEE33FEE54E2FF582E54D81
:106F15001254F7926720670B054FC3E54F648094C1
:0B6F25009040CBC22BC22CC22DC22E0C
:016F3000223E
:0472E3008C4D8D4EF3
:1072E700EF6038E4F54F854E82854D83E0FEA3E0DD
:1072F7004E6028AF4FEF3395E0FEEF25E0FFEE330A
:10730700FEE54E2FF582E54D1254F7926720670B85
:0B731700054FC3E54F6480949040CB0D
:017322002248
:0854F7003EF583E0FEA3E0FF97
:0454FF00AD07AC0643
:10550300C268780CEF088006A2E0CE13CE13D8F859
:10551300540FF5507808AF05AE04EF088006A2E0FB
:10552300CE13CE13D8F8540FF5517804AF05AE045B
:10553300EF088006A2E0CE13CE13D8F8540FF5522D
:10554300ED540FF553E550607CB4010BAB53AD52F2
:10555300AF5112581E806EE550B4030BAB53AD52DE
:10556300AF51126A82805EE550B4040BAB53AD5267
:10557300AF51126ADF804EE550B4050BAB53AD5209
:10558300AF51123CEE803EE550B4060BAB53AD5227
:10559300AF5112180F802EE550B4070BAB53AD5229
:1055A300AF51125422801EE550B4080BAB53AD52D9
:1055B300AF51126E8F800EE550B40909AB53AD5253
:0755C300AF5112787CA268D1
:0155CA0022BE
:10581E008F548D558B56E554B40113900020E0FF44
:10582E00126A2A900020EFF0FD7F200258B9E5544D
:10583E00B40211900021126A24900021EFF0FD7F36
:10584E00210258B9E554B40310900022126A249034
:10585E000022EFF0FD7F228052E554B40410900038
:10586E0023126A24900023EFF0FD7F23803DE55440
:10587E00B40510900024126A24900024EFF0FD7FEE
:10588E00248028E554B40610900025126A24900056
:10589E0025EFF0FD7F258013E554B4071390002605
:1058AE00126A24900026EFF0FD7F267E00027323FD
:1058BE00E554B40816900027126A24900027EFF0E2
:0C58CE00FD7F277E0012732312766A22F1
:066A2400E0FFAB56AD558A
:106A2A00D269AC07BD01047E018033BD02047E0237
:106A3A00802CBD03047E048025BD04047E08801ECC
:106A4A00BD05047E108017BD06047E208010BD0798
:106A5A00047E408009BD08047E808002C269BB01B1
:106A6A0005EE4204800BEB7006EEF452048002C27B
:076A7A0069306903AF04223B
:016A810022F2
:106A82008F548D558B56E554700BAD56AF55127B16
:106A920054E4FD801EE554B4010BAD56AF55127B94
:106AA200547D01800EE554B4020CAD56AF55127BF5
:106AB200547D02023861E554B4030CE5557008D2E6
:106AC20069127218C25822E554B40410AD56AF557B
:0D6AD2001267268F3F753D05E53D70FC22E3
:106ADF008F548D558B56E5547036E555B40108E546
:106AEF005614FF7D018026E555B40208E55614FFC4
:106AFF007D028019E555B40308E55614FF7D038028
:106B0F000CE55564047022E55614FF7D040271D222
:106B1F00E554B40114E555D39400400DE5559405A3
:0A6B2F005007753D01E53D70FC22A2
:103CEE008B54EF7017BD0114E5547002C220E554D9
:103CFE0064016003023E5AD220023E5AEF7017BD95
:103D0E000214E5547002C221E55464016003023EC0
:103D1E005AD221023E5AEF7017BD0314E5547002B9
:103D2E00C222E55464016003023E5AD222023E5A78
:103D3E00EF7017BD0414E5547002C223E5546401FC
:103D4E006003023E5AD223023E5AEF701BBD051885
:103D5E00E5547004C220C221E55464016003023EA2
:103D6E005AD220D221023E5AEF701BBD0618E554DE
:103D7E007004C222C223E55464016003023E5AD28B
:103D8E0022D223023E5ABF0117BD0114E554700220
:103D9E00C224E55464016003023E5AD224023E5A04
:103DAE00BF0117BD0214E5547002C225E55464012B
:103DBE006003023E5AD225023E5ABF0116BD0313BE
:103DCE00E5547002C226E55464016003023E5AD2E5
:103DDE00268079BF0113BD0410E5547002C227E599
:103DEE005464017067D2278063BF0117BD0514E5C7
:103DFE00547004C224C225E5546401704FD224D2FB
:103E0E00258049BF0117BD0614E5547004C226C2B1
:103E1E0027E55464017035D226D227802FEF640136
:103E2E00702AED64097025E554B401047F018019F0
:103E3E00E554B402047F028010E554B403047F03FA
:103E4E008007E554B404057F04126BEC7F327E00CC
:043E5E00127A15229D
:10180F008F548D558B56E5547016AD56AF55127BD0
:10181F0054901D14EFF0901D14E0D3940050F72254
:10182F00E554B40117E555B40112E5567002C2082C
:10183F00E55664016003021BB5D20822E554B401DA
:10184F0017E555B40212E5567002C209E556640158
:10185F006003021BB5D20922E554B40117E555B454
:10186F000312E5567002C20EE55664016003021BB7
:10187F00B5D20E22E554B40117E555B40412E5565E
:10188F007002C20CE55664016003021BB5D20C2234
:10189F00E554B4011BE555B40516E5567004C208AE
:1018AF00C209E55664016003021BB5D208D20922B2
:1018BF00E554B40118E555B40613E5567004C20E8D
:1018CF00C20CE55664016003021BB58024E5546425
:1018DF00017023E555B4071EE5567008C208C2090A
:1018EF00C20EC20CE55664016003021BB5D208D2CA
:1018FF0009D20ED20C22E554B4021DE555B40118DD
:10190F00E5567004C208C220E55664016003021B4D
:10191F00B5D208D220021AD5E554B4021DE555B44C
:10192F000218E5567004C209C221E556640160032E
:10193F00021BB5D209D221021A61E554B4021DE58A
:10194F0055B40318E5567004C20EC222E556640161
:10195F006003021BB5D20ED222021A85E554B402DF
:10196F001DE555B40418E5567004C20CC223E556A4
:10197F0064016003021BB5D20CD223021AA8E554EE
:10198F0064027026E55564057020E5567008C2089C
:10199F00C209C220C221E55664016003021BB5D201
:1019AF0008D209D220D221021AD5E554640270263A
:1019BF00E55564067020E5567008C20EC20CC222AF
:1019CF00C223E55664016003021BB5D20ED20CD2BE
:1019DF0022D223021A85E55464027035E555640757
:1019EF00702FE5567010C208C209C20EC20CC22079
:1019FF00C221C222C223E55664016003021BB5D285
:101A0F0008D209D20ED20CD220D221D222D22380D8
:101A1F0065E554B4031DE555B40118E5567004C2CD
:101A2F0008C224E55664016003021BB5D208D22414
:101A3F00021AD5E554B4031FE555B4021AE55670E2
:101A4F0004C209C225E55664016003021BB5D20921
:101A5F00D2257F02021B04E554B4031EE555B403DF
:101A6F0019E5567004C20EC226E5566401600302E2
:101A7F001BB5D20ED2267F03807BE554B4031EE53F
:101A8F0055B40419E5567004C20CC227E55664011B
:101A9F006003021BB5D20CD2277F048058E5546433
:101AAF00037027E55564057021E5567008C208C21A
:101ABF0009C224C225E55664016003021BB5D20892
:101ACF00D209D224D2257F01802BE55464037028DC
:101ADF00E55564067022E5567008C20EC20CC22688
:101AEF00C227E55664016003021BB5D20ED20CD299
:101AFF0026D2277F03026BECE554B4040AE555B4F4
:101B0F000105AF56026665E554B4040AE555B40203
:101B1F0005AF5602689FE5546409701EE555B40180
:101B2F0019E5567003C20A22E556B40103D20A2200
:101B3F00E556640270707F058069E5546409701E74
:101B4F00E555B40219E5567003C20B22E556B401F0
:101B5F0003D20B22E5566402704C7F068045E55494
:101B6F006409701EE555B40319E5567003C20F22C0
:101B7F00E556B40103D20F22E556640270287F07A1
:101B8F008021E5546409701EE555B40419E55670BB
:101B9F0003C20D22E556B40103D20D22E556B4025D
:071BAF00057F081260A72268
:10542200AC07EC60030254D8BD010CEB700990008C
:105432001FE054FDF0800DBD010ABB010790001F63
:10544200E04403F0BD020CEB700990001FE054FB36
:10545200F0800DBD020ABB010790001FE04405F079
:10546200BD030CEB700990001FE054F7F0800DBDF6
:10547200030ABB010790001FE04409F0BD040CEBD6
:10548200700990001FE054F9F0800DBD040ABB01C1
:105492000790001FE04407F0BD050CEB7009900077
:1054A2001FE054F3F0800DBD050ABB010790001FF9
:1054B200E0440DF0BD060CEB700990001FE054F1C2
:1054C200F08025ED64067020EB6401701B90001FD4
:1054D200E0440FF08012BC010FED700CEB7004C2BF
:1054E200298005BB0102D22990001FE0FD7F1F7EAB
:0554F2000012732322EB
:106E8F008F548D558B56E554700C127B50744F2FC9
:106E9F00F58274068020E554B4010C127B50744FB8
:106EAF002FF58274068024E554B40210127B5074BF
:106EBF009F2FF58274063EF583E4F022E554B40368
:106ECF0010127B50749F2FF58274063EF583740168
:026EDF00F0229F
:02787C008F5427
:10787E00AF057804EF08800123D8FD4BF555E5548C
:10788E00B40908E555B49903026011AD55AF541211
:02789E0076EE84
:0178A00022C5
:10666500E545B40109BF0106D220D2088060E545A1
:10667500B40109EF7006C220C2088052E545B40294
:1066850009BF0106D221D2098044E545B40209EFCC
:106695007006C221C2098036E545B40309BF01066B
:1066A500D222D20E8028E545B40309EF7006C22236
:1066B500C20E801AE545B40409BF0106D223D20CE7
:1066C500800CE545B40407EF7004C223C20C1279AF
:0A66D500F9AF3E126BEC1279DD22E2
:10689F00E545B40108BF0105D224D20822E545B46D
:1068AF000108EF7005C224C20822E545B40208BFF3
:1068BF000105D225D20922E545B40208EF7005C2C1
:1068CF0025C20922E545B40308BF0105D226D20E21
:1068DF0022E545B40308EF7005C226C20E22E54536
:1068EF00B40408BF0105D227D20C22E545B4040732
:0868FF00EF7004C227C20C2255
:047B5000AD56AF552A
:0D7B5400EF75F00AA47C002DFFEC35F0FE6B
:017B61002201
:020941008F4DD8
:10094300C268E4F53DD25ED26B125A497D4B7F02F9
:100953001276EE7D04E4FF1276EE7D387F04127684
:10096300EE7D607F021276EE90061CE0FFA3E0901E
:100973001CE8CFF0A3EFF0C26BAF4D125A49E4F578
:1009830046C208123346E54DB40106A24992678078
:100993001FE54DB40206A24D92678014E54DB403E2
:1009A30006A25192678009E54DB40404A2549267EC
:1009B300901CE8E07002A3E07005D268020F8B3050
:1009C30067C1123346E54DB40106A2499267801F01
:1009D300E54DB40206A24D92678014E54DB40306BB
:1009E300A25192678009E54DB40404A25492672092
:1009F30067D0E54DB4010A754E1B754F10786880BA
:100A03002BE54DB4020A754E1B754F607869801C47
:100A1300E54DB4030A754E1B754FB0786A800DE53A
:100A23004DB4040B754E1C754F00786BE6F550E51D
:100A330050D394005003020F85854F82854E83E087
:100A4300640B6003020F80A3E0FFB40A0AE550B40D
:100A53000205D268020F85EF64017032854F8285EB
:100A63004E83A3A3E064037025E550B40520854FAE
:100A730082854E83A3A3A3E0FFE54F2404F582E41C
:100A8300354EF583E0FDAB4D123FBC020F85854F1C
:100A930082854E83A3E0B40121854F82854E83A3D3
:100AA300A3E0B40415E550D39405400EAB4DAD4F10
:100AB300AC4EAF50123510020F85854F82854E83A1
:100AC300A3E064017032854F82854E83A3A3E06463
:100AD300057025E550B40520854F82854E83A3A379
:100AE300A3E0FFE54F2404F582E4354EF583E0FDF2
:100AF300AB4D126569020F85854F82854E83A3E056
:100B030064017032854F82854E83A3A3E06406702F
:100B130025E550B40520854F82854E83A3A3A3E02A
:100B2300FFE54F2404F582E4354EF583E0FDAB4D3C
:100B3300125C58020F85854F82854E83A3E0B40172
:100B430021854F82854E83A3A3E0B40715E550D3D7
:100B53009405400EAB4DAD4FAC4EAF50124CAD02B1
:100B63000F85854F82854E83A3E064017032854FE4
:100B730082854E83A3A3E064087025E550B4052065
:100B8300854F82854E83A3A3A3E0FFE54F2404F59D
:100B930082E4354EF583E0FDAB4D126B39020F85D0
:100BA300854F82854E83A3E0B40219854F82854E1B
:100BB30083A3A3E0B4080DE550B40308AF4D127648
:100BC300C2020F85854F82854E83A3E064027024A1
:100BD300854F82854E83A3A3E0B40818E550B4047F
:100BE30013854F82854E83A3A3A3E0FFAD4D1277F8
:100BF300BB020F85854F82854E83A3E0B40219851E
:100C03004F82854E83A3A3E0B4090DE550B40308D6
:100C1300AF4D127696020F85854F82854E83A3E0F2
:100C230064027024854F82854E83A3A3E0B4091820
:100C3300E550B40413854F82854E83A3A3A3E0FF3D
:100C4300AD4D127793020F85854F82854E83A3E0C6
:100C530064037036854F82854E83A3A3E0640A70D4
:100C630029E55064057023854F82854E83A3A3A392
:100C7300E0FFE54F2404F582E4354EF583E0FD12F1
:100C830079AEAD4D12575F020F85854F82854E8336
:100C9300A3E06403703E854F82854E83A3A3E06483
:100CA300017031E550D39405402A854F82854E83E8
:100CB300A3A3A3E0FFE54F2404F582E4354EF583B7
:100CC300E0FD1279AE854D55AB50AD4FAC4E12469B
:100CD30070020F85854F82854E83A3E064037036CF
:100CE300854F82854E83A3A3E064027029E5506497
:100CF300057023854F82854E83A3A3A3E0FFE54FB1
:100D03002404F582E4354EF583E0FD1279AEAD4D52
:100D13001270B0020F85854F82854E83A3E0B40322
:100D230019854F82854E83A3A3E0B4030DE550B428
:100D33000308AF4D127361020F85854F82854E8381
:100D4300A3E0B40321854F82854E83A3A3E0B404BB
:100D530015E550D39403400EAB4DAD50AF4FAE4E9F
:100D6300125EE0020F85854F82854E83A3E0B403B4
:100D730019854F82854E83A3A3E0B4050DE550B4D6
:100D83000308AF4D127B62020F85854F82854E8328
:100D9300A3E0B4031D854F82854E83A3A3E0B4066D
:100DA30011E550B4050CAD4DAF4FAE4E1273DA02E0
:100DB3000F85854F82854E83A3E064037024854F9E
:100DC30082854E83A3A3E0B40718E550B4041385CA
:100DD3004F82854E83A3A3A3E0FFAD4D1279280272
:100DE3000F85854F82854E83A3E0B4031D854F8213
:100DF300854E83A3A3E0B40811E550B4050CAD4DB3
:100E0300AF4FAE4E1275B0020F85854F82854E836C
:100E1300A3E064057022E550B4041D854F82854E1E
:100E230083A3A3E0FF854F82854E83A3A3A3E0FDA5
:100E3300AB4D122D80020F85854F82854E83A3E033
:100E4300B40524E54F2404F582E4354EF583E0B47C
:100E53000B15E550D39405400EAB4DAD50AF4FAEDF
:100E63004E124780020F85854F82854E83A3E0642F
:100E7300067022E550B4041D854F82854E83A3A3DB
:100E8300E0FF854F82854E83A3A3A3E0FDAB4D1204
:100E9300267D020F85854F82854E83A3E0B4062409
:100EA300E54F2404F582E4354EF583E0B40B15E5F4
:100EB30050D39405400EAB4DAD50AF4FAE4E1231F3
:100EC3005E020F85854F82854E83A3E064097022FD
:100ED300854F82854E83A3A3E0B40A16E550B4047C
:100EE30011854F82854E83A3A3A3E0FF12701B02DB
:100EF3000F85854F82854E83A3E064097023854F58
:100F030082854E83A3A3E0B40117E550B404128590
:100F13004F82854E83A3A3A3E0FFAD4D12569B8062
:100F230061854F82854E83A3E0B40920854F828576
:100F33004E83A3A3E0B40214E550D39404400DAB55
:100F430050AD4DAF4FAE4E1214648036854F82853F
:100F53004E83A3E064097025854F82854E83A3A346
:100F6300E0B40317E550B40412854F82854E83A382
:100F7300A3A3E0FFAD4D126F3180078000AF4D1288
:100F830079C0206803020986C258D26BAF4D125A4A
:100F9300497D607F021276EE7D327F031276EEC2C8
:0F0FA3006BAF4D125A49126FD0E4786CF6C25EF4
:010FB200221C
:083510008F518C528D538B5436
:10351800855382855283A3A3A3E0FF8D828C83E524
:1035280082240412671D8F55E555D3940050030279
:1035380036B1E555942940030236B1E55164067069
:103548004FD26BAF54125A497D527F051276EEAFB7
:1035580055124BABE5532405F582E43552F583E06B
:10356800B40112749F2555F582E43406F58374017D
:10357800F07D38800F749F2555F582E43406F58375
:10358800E4F07D367F061276EEC26BAF54025A49DC
:10359800E5532406F582E43552F583E0640B6003B5
:1035A8000236B1E5532405F582E43552F583E0B4DB
:1035B8000110749F2555F582E43406F5837401F0F3
:1035C800800D749F2555F582E43406F583E4F0E414
:1035D800FFFEE5532407F582E43552F583E5822E94
:1035E800F582E43583F583E0B40B04AF0680040E5E
:1035F800BE08DFEF70030236B1C3940840030236F9
:10360800B175F008E555A424F8F582E5F03400F525
:1036180083EFF07E01EF2401FDE433FCEEC39DEC63
:103628006480F87480985036E5532406F582E435B2
:1036380052F583E5822EF582E43583F583E0FD7546
:10364800F008E555A424F8F582E5F03400F583E5A3
:10365800822EF582E43583F583EDF00E80B7E553CD
:103668002408F582E43552F583E5822FF582E435A6
:1036780083F583E0640B602DEF2408FEC3E5519EBB
:10368800F55175F0041258DAAEF0EE701CE55324CB
:1036980007FDE43552FC7E00ED2FFBEE3CFAAD55FC
:1036A8007F011239ECD26A8002C26AAF54127B944D
:0136B80022EF
:1078C5008E5CF55DAF5BEF3395E0FEE5592FF582F4
:0878D500E5583EF583A3E0FF36
:0A78DD00EFD3940940037F0022223C
:0839EC008F568D578A588B5944
:1039F400755B01E4F55AAF5BEF3395E0FEE5592FB3
:103A0400F582E5583EF583E0FF640970651278DDC0
:103A1400755C008F5DAE5C7804EF08800633CE33AE
:103A2400CE92E0D8F81278C5EF425DAE5CAF5D7817
:103A340008EF08800633CE33CE92E0D8F88E5CF5DA
:103A44005DAF5BEF3395E0FEE5592FF582E5583E17
:103A5400F583A3A3E0FFE55BFD3395E0FCE5592D79
:103A6400F582E5583CF583A3A3A3E0FD1279AE02E9
:103A74003B07AF5BEF3395E0FEE5592FF582E55840
:103A84003EF583E0FF1278DD755C008F5DAE5C78F7
:103A940004EF08800633CE33CE92E0D8F81278C50E
:103AA400EF425DAE5CAF5D7804EF08800633CE3341
:103AB400CE92E0D8F88E5CF55DAF5BEF3395E0FE17
:103AC400E5592FF582E5583EF583A3A3E0FF12786C
:103AD400DDEF425DAE5CAF5D7804EF08800633CE67
:103AE40033CE92E0D8F88E5CF55DAF5BEF3395E0B2
:103AF400FEE5592FF582E5583EF583A3A3A3E0FF25
:103B04001278DDEF425DE556701EAF5AEF3395E053
:103B1400FEEF25E0FFEE33FE75F020E557A424D038
:103B2400F582E5F034068021E556B4012FAF5AEF53
:103B34003395E0FEEF25E0FFEE33FE75F020E55708
:103B4400A424D0F582E5F03410F583E5822FF582C4
:103B5400E5833EF583E55CF0A3E55DF07404255B45
:103B6400F55B055AC3E55A6480949050030239FA10
:013B7400222E
:084CAD008F518C528D538B5482
:104CB500855382855283A3A3A3E0FF8D828C83E570
:104CC50082240412671D8F55E555D39400500302C5
:104CD5004D9AE55594334003024D9AE551640670AB
:104CE5004FD26BAF54125A497D527F051276EEAF03
:104CF50055124BABE5532405F582E43552F583E0B7
:104D0500B40112744F2555F582E43406F583740118
:104D1500F07D38800F744F2555F582E43406F58310
:104D2500E4F07D367F061276EEC26BAF54025A4927
:104D3500E5532406F582E43552F583E0640B70559E
:104D4500E5532405F582E43552F583E0B40110748A
:104D55004F2555F582E43406F5837401F0800D7412
:104D65004F2555F582E43406F583E4F074F92551B1
:104D7500F55175F0041258DAAFF0EF7014E55324CD
:104D850006FBE43552FAAD55E4FF1239ECD26A80E0
:104D95000DC26A8009C26BAF54125A49C26AAF5438
:034DA500127B94EA
:014DA80022E8
:023FBC008B5127
:103FBE001267268F54E554D394005003024100E556
:103FCE005494334003024100D26BAF51125A497DD3
:103FDE00527F051276EEAF54124BAB749F2554F5FB
:103FEE0082E43406F583E060047D3880027D367FFE
:103FFE00061276EE7F2C7E01127A1575F008E554C6
:10400E00A424F8F582E5F03400F583E0F55270074C
:10401E007D1B7F061276EE7D577F021276EEE552FD
:10402E0070030240B1755301AF52EF3395E0FEEFCE
:10403E002401FFE43EFEAD53ED3395E0FCC3ED9F4E
:10404E00EE6480F8EC6480985059AF53EF3395E0EE
:10405E00FE75F008E554A424F8F582E5F03400F579
:10406E0083E5822FF582E5833EF583E0FFD3940945
:10407E00400512725D8028AF53EF3395E0FE75F068
:10408E0008E554A424F8F582E5F03400F583E582C2
:10409E002FF582E5833EF583E0FDE4FF1276EE0513
:1040AE005380857F2C7E01127A1575F020E554A47D
:1040BE0024D0F582E5F03410F583E0FEA3E0FF9006
:1040CE000000EEF0A3EFF04E70077D1B7F06127618
:1040DE00EE7D0C7F031276EE900000E07002A3E0FE
:1040EE006009E55414FD7F01122F74C26BAF5102AB
:0940FE005A49C26AAF51127B94C9
:014107002295
:042F74008F558D5692
:102F7800E4F557E555600302301FAF57EF3395E08E
:102F8800FEEF25E0FDEE33FCAF56EF3395E0FEEFA4
:102F98007805C333CE33CED8F924F0F58274063ED3
:102FA800F583E5822DF582E5833CF583E0FAA3E01D
:102FB800FB780CFFAE02088006A2E0CE13CE13D831
:102FC800F8540FF5587808AF03AE02EF088006A250
:102FD800E0CE13CE13D8F8540FF559AF56EF33950A
:102FE800E0FEEF7805C333CE33CED8F924F0F5826E
:102FF80074063EF583E5822DF582E5833CF583E092
:10300800FCA3E0FD7804FFAE04088006A2E0CE131E
:10301800CE13D8F80230C2E555640160030230CB04
:10302800AF57EF3395E0FEEF25E0FDEE33FCAF56EA
:10303800EF3395E0FEEF7805C333CE33CED8F924CD
:10304800F0F58274103EF583E5822DF582E5833C28
:10305800F583E0FAA3E0FB780CFFAE02088006A235
:10306800E0CE13CE13D8F8540FF5587808AF03AE56
:1030780002EF088006A2E0CE13CE13D8F8540FF55D
:1030880059AF56EF3395E0FEEF7805C333CE33CE14
:10309800D8F924F0F58274103EF583E5822DF58287
:1030A800E5833CF583E0FCA3E0FD7804FFAE04086B
:1030B8008006A2E0CE13CE13D8F8540FF55AED547B
:1030C8000FF55BE558700FE559700BE55A7007E589
:1030D8005B700302315DAD58E4FF1276EEAD59E442
:1030E800FF1276EEE55864097048855A5CAF5CFEBD
:1030F8007804EF08800633CE33CE92E0D8F8F55C3A
:10310800E55B425CE55CB4990B7D09E4FF1276EE61
:103118007D098027E55C75F00A84F55DFDE4FF1202
:1031280076EEE55D75F00AA4FFC3E55C9FF55DFDED
:103138008009AD5AE4FF1276EEAD5BE4FF1276EE3D
:103148007FF47E01127A150557C3E557648094A071
:053158005003022F7B73
:01315D00224F
:025C58008B516E
:105C5A001267268F52E552D394005003025CF4E592
:105C6A005294334003025CF4D26BAF51125A497D0D
:105C7A00527F051276EEAF52124BAB744F2552F596
:105C8A0082E43406F583E060047D3880027D367F45
:105C9A00061276EE7F2C7E01127A157F2C7E011277
:105CAA007A1575F020E552A424D0F582E5F0340681
:105CBA00F583E0FEA3E0FF900000EEF0A3EFF04EC4
:105CCA0070077D1B7F061276EE7D0C7F031276EE3F
:105CDA00900000E07002A3E06009E55214FDE4FFC1
:105CEA00122F74C26BAF51025A49C26AAF51127B6A
:015CFA009415
:015CFB002286
:026569008B5154
:10656B00126726AD07EDD39400406BED9433506664
:10657B00E4FCECFF3395E0FEEF25E0FFEE33FE7518
:10658B00F020EDA424D0F582E5F03410F583E582FC
:10659B002FF582E5833EF583E4F0A3F00CBC10D21B
:1065AB00749F2DF582E43406F583E4F0FCECFF33A5
:1065BB0095E0FE75F008EDA424F8F582E5F03400C3
:1065CB00F583E5822FF582E5833EF583E4F00CBC81
:0D65DB0008DBD26A8002C26AAF51127B94C5
:0165E8002290
:026B39008B517E
:106B3B00126726AD07EDD394004045ED94335040DA
:106B4B00E4FCECFF3395E0FEEF25E0FFEE33FE7542
:106B5B00F020EDA424D0F582E5F03406F583E58230
:106B6B002FF582E5833EF583E4F0A3F00CBC10D245
:106B7B00744F2DF582E43406F583E4F0D26A80027B
:076B8B00C26AAF51127B94B6
:016B920022E0
:10751A002430F58274003EF583EDF0AF55EF3395D4
:10752A00E0FEE5522FF582E5513EF583A3A3E0FF85
:10753A00D3EF648094814008EF6480948A500122DA
:03754A007F00229D
:107B3D00D3EF648094804008EF648094A1500122BB
:037B4D007F002294
:081464008E518F528D538B5401
:10146C008F828E83A3A3A3E014F55674FC2554F548
:10147C00546403600FE55464076009E554640B6021
:10148C0003021807C3E556648094805003021807C2
:10149C00E556648094884003021807E4F555AF566E
:1014AC00EF3395E0FEEF7803C333CE33CED8F92477
:1014BC0030F58274003EF583AF55EF3395E0FEE5D1
:1014CC00822FF582E5833EF583E4F00555E555B4AE
:1014DC0008CC755504E5546403705FAF55EF339534
:1014EC00E0FEE5522FF582E5513EF583E0FFE55530
:1014FC00FD3395E0FCE5522DF582E5513CF583A3D7
:10150C00E0FD126726127B3DAD07AF56EF3395E039
:10151C00FEEF7803C333CE33CED8F912751AAD076C
:10152C00AF56EF3395E0FEEF7803C333CE33CED80E
:10153C00F92431F58274000217FEE5546407600348
:10154C00021639AF55EF3395E0FEE5522FF582E5E3
:10155C00513EF583E0FFE555FD3395E0FCE5522D5A
:10156C00F582E5513CF583A3E0FD126726127B3D25
:10157C00AD07AF56EF3395E0FEEF7803C333CE33B0
:10158C00CED8F912751AAD07AF56EF3395E0FEEFD2
:10159C007803C333CE33CED8F92431F58274003EB0
:1015AC00F583EDF0AF55EF3395E0FEE5522FF58264
:1015BC00E5513EF583A3127536AD07AF56EF339563
:1015CC00E0FEEF7803C333CE33CED8F91266DF12C8
:1015DC007B3DAD07AF56EF3395E0FEEF7803C33399
:1015EC00CE33CED8F92433F58274003EF583EDF07A
:1015FC00AF55EF3395E0FEE5522FF582E5513EF500
:10160C0083E5822406F582E43583F583E0FF1275C9
:10161C003AAD07AF56EF3395E0FEEF7803C333CE08
:10162C0033CED8F92434F58274000217FEE55464E5
:10163C000B6003021807AF55EF3395E0FEE5522F10
:10164C00F582E5513EF583E0FFE555FD3395E0FC71
:10165C00E5522DF582E5513CF583A3E0FD1267269A
:10166C00127B3DAD07AF56EF3395E0FEEF7803C329
:10167C0033CE33CED8F912751AAD07AF56EF33957A
:10168C00E0FEEF7803C333CE33CED8F92431F582A4
:10169C0074003EF583EDF0AF55EF3395E0FEE55267
:1016AC002FF582E5513EF583A3127536AD07AF5683
:1016BC00EF3395E0FEEF7803C333CE33CED8F91277
:1016CC0066DF127B3DAD07AF56EF3395E0FEEF784A
:1016DC0003C333CE33CED8F92433F58274003EF5F0
:1016EC0083EDF0AF55EF3395E0FEE5522FF582E533
:1016FC00513EF583E5822406F582E43583F583E0DB
:10170C00FF12753AAD07AF56EF3395E0FEEF780355
:10171C00C333CE33CED8F92434F58274003EF5832E
:10172C00EDF0AF55EF3395E0FEE5522FF582E55124
:10173C003EF583E5822407F582E43583F583E0FFEB
:10174C0012753AAD07AF56EF3395E0FEEF7803C351
:10175C0033CE33CED8F92435F58274003EF583EDC3
:10176C00F0AF55EF3395E0FEE5522FF582E5513E93
:10177C00F583E5822408F582E43583F583E0FFE503
:10178C0055FD3395E0FCE5522DF582E5513CF58392
:10179C00E582240912671D127B3DAD07AF56EF336E
:1017AC0095E0FEEF7803C333CE33CED8F92436F56B
:1017BC008274003EF583EDF0AF55EF3395E0FEE516
:1017CC00522FF582E5513EF583E582240AF582E439
:1017DC003583F583E0FF12753AAD07AF56EF3395BD
:1017EC00E0FEEF7803C333CE33CED8F92437F5823D
:1017FC0074003EF583EDF0D26A8002C26AAF5312D8
:02180C007B94CB
:01180E0022B7
:10701B00EF24FE601014601314601624037016D254
:10702B0008D2248010D209D225800AD20ED2268013
:10703B0004D20CD2277FF47E01127A15753D04E53C
:10704B003D70FC7F647E00127A15C224C225C226D5
:0B705B00C227C208C209C20EC20C22EC
:04569B008D51AC077A
:10569F00C3EC64809481500302575EEC648094895C
:1056AF00400302575EE4F552AF51EF3395E0FEEF42
:1056BF007803C333CE33CED8F924E8F582741A3E7B
:1056CF00F583AF52EF3395E0FEE5822FF582E58348
:1056DF003EF583E0FD74182FF582741D3EF583EDC2
:1056EF00F00552E552B408C0EC14FFAD511271D25F
:1056FF00D269AF51125AFD753D017F327E00127A89
:10570F0015E53D70FCC269AF51125AFDE4F552E543
:10571F0052FD3395E0FC74182DF582741D3CF58312
:10572F00E0FBAF51EF3395E0FEEF7803C333CE3399
:10573F00CED8F924E8F582741A3EF583E5822DF56B
:0F574F0082E5833CF583EBF00552E552B408C0C8
:01575E002228
:046F31008D51AC07CB
:106F3500D3EC64809480403CEC648094895035E4C3
:106F4500FDECFF3395E0FEEF7803C333CE33CED8A7
:106F5500F92428F58274003EF583EDFF3395E0FEB4
:106F6500E5822FF582E5833EF583E4F00DBD08D17A
:0B6F7500D26A8002C26AAF51127B9406
:016F800022EE
:044670008C528D5388
:10467400D3EF648094805003024778EF648094956C
:104684004003024778EB648094875003024778EB39
:10469400648094E44003024778EF3395E0FEEF78BA
:1046A40005C333CE33CED8F92460F58274033EAF0C
:1046B40082F5568F57EB24FBF558D394025003022E
:1046C4004778E55875F00384E5F06003024778E520
:1046D4005875F00384F55AC39410400302477805D3
:1046E40057E557AE567002055614F5828E83E55A87
:1046F400F074052553F553E43552F552E4F558E5C5
:1047040058C3955A506A855382855283E0F559B44B
:104714000A130557E557AE567002055614F5828EF6
:1047240083E4F080120557E557AE5670020556141F
:10473400F5828E83E559F0855382855283A3E0FF89
:10474400855382855283A3A3E0FD1279AE8F590568
:1047540057E557AE567002055614F5828E83E55917
:10476400F074032553F553E43552F5520558808F00
:0B477400D26A8002C26AAF55127B942B
:01477F002217
:04575F008F518D5287
:10576300E551D394005003025816E55194154003B4
:10577300025816D26BAF52125A497D5F7F051276DB
:10578300EEAD51E4FF1276EE7D527F041276EE7F8A
:10579300F47E01127A1575F020E551A42460F58298
:1057A300E5F03403AF82F5558F56F583E0F553608A
:1057B3004DD394004056E55394105050E55325E0E3
:1057C300F553755401E5532401FFE433FEC3E55457
:1057D3009FEE6480F87480985032E5562554F58224
:1057E300E43555F583E0FFE5562554F582E4355558
:1057F300F583A3E0FD1276EE0554055480C77D1BA7
:105803007F061276EE7D5F7F051276EEC26BAF5296
:0A581300025A49C26AAF52127B9498
:01581D002268
:107793008D51EFD3940A4006EFD3940F4003EF705B
:1077A3000E90063FEFF0D26AAF51127B94D322C200
:0877B3006AAF51127B94C3225E
:1077BB008D51EFD3940A4006EFD3940F4003EF7033
:1077CB000E90063BEFF0D26AAF51127B94D322C2DC
:0877DB006AAF51127B94C32236
:10725D008F55E555B40B067D5F7F078034E555B43A
:10726D000C067D5E7F068029E555B40D067D0A7FEF
:10727D0002801EE555B40E067D327F028013E55562
:10728D00B40F067D467F028008E55570077D0A7FA5
:05729D00031276EE2251
:107696008F51D26B125A497D207F051276EE7D2ED0
:1076A6007F031276EE7D527F041276EE90063FE05F
:0C76B600FF12725DC26BAF51125A4922E4
:1076C2008F51D26B125A497D207F051276EE7D21B1
:1076D2007F061276EE7D527F041276EE90063BE034
:0C76E200FF12725DC26BAF51125A4922B8
:107928008D51D3EF64809480400EEF64809486502C
:107938000712747ED26A8002C26AAF51127B942207
:0673DA008D51AB07AA066D
:1073E0008B828A83A3A3A3E0FFEB2404F582E43A13
:1073F000126722D3EF648094804010EF648094A1E0
:10740000500990063DEFF0D26A8002C26AAF511275
:027410007B946B
:017412002257
:0675B0008D51AB07AA0695
:1075B6008B828A83A3A3A3E0FFEB2404F582E43A3B
:1075C600126722EFC39421500990063CEFF0D26A6D
:0975D6008002C26AAF51127B94DD
:0175DF002289
:065EE0008E518F528B531E
:105EE600755406755540D3ED64809484407CED640A
:105EF6008094A55075ED24FDF556D39404406BE5CA
:105F06005620E06613F5570555E555AE5470020563
:105F16005414F5828E83E557F074032552F552E446
:105F26003551F551E4F556E556C39557503385522C
:105F360082855183E0FFA3E0FD1279AE0555E55554
:105F4600AC547002055414F5828C83EFF00552E5CB
:105F560052700205510552E55270020551055680F0
:105F6600C6D26AAF53127B94D322C26AAF53127B56
:025F760094C3D2
:015F78002206
:084780008E518F528D538B54B2
:10478800C269D3E553648094845003024835E553E5
:104798006480948D40030248358F828E83A3A3E002
:1047A800640A60030248358F828E83A3A3A3E014B2
:1047B800B4080050769047CB75F003A4C58325F064
:1047C800C583730247E30247ED0247F70248010237
:1047D800480B02481502481F0248297555007556AE
:1047E80080D2698048755500755688D269803E75B3
:1047F8005500755690D2698034755500755698D213
:1048080069802A7555007556A0D2698020755500B3
:104818007556A8D26980167555007556B0D269804C
:104828000C755500755678D2698002C26930695096
:10483800E4FFEF7C002556FDEC35558D82F583E4C9
:10484800F00FBF08EDE55324FB855682855583F0AC
:104858007F01E5522404F582E43551F583E5822F82
:10486800F582E43583F583E0FEEF7C002556FDEC08
:1048780035558D82F583EEF00FBF08D6D26A8002D7
:07488800C26AAF54127B94D9
:01488F002206
:0461C8008E548F550D
:1061CC000555E5557002055414F5828E83E0F5579C
:1061DC006074C39408506F7F2C7E01127A15E4F51D
:1061EC0056E556C39557505E855582855483E060BD
:1061FC003624F5601414601714601A14601D1460B2
:10620C002024057028E4FD802D7D5F7F0780287D8C
:10621C005E7F0680227D0A7F02801C7D327F028099
:10622C00167D467F0280107D0A7F03800A85558289
:10623C00855483E0FDE4FF1276EE0555E5557002BA
:06624C0005540556809B7D
:016252002229
:022D80008B5175
:102D8200C269EF640A6003022F5BED14B4080040CD
:102D920003022F59902DA475F003A4C58325F0C515
:102DA2008373022DBC022DF0022E24022E58022E15
:102DB2008C022EC0022EF3022F26D26BAF51125A72
:102DC200497D577F021276EE7D05E4FF1276EEE42E
:102DD200FDFF1276EE7D01E4FF1276EE7D527F0456
:102DE2001276EE755200755380D269022F5BD26B58
:102DF200AF51125A497D577F021276EE7D05E4FFEC
:102E02001276EEE4FDFF1276EE7D02E4FF1276EE1C
:102E12007D527F041276EE755200755388D2690294
:102E22002F5BD26BAF51125A497D577F021276EE59
:102E32007D05E4FF1276EEE4FDFF1276EE7D03E4FB
:102E4200FF1276EE7D527F041276EE7552007553B4
:102E520090D269022F5BD26BAF51125A497D577FD4
:102E6200021276EE7D05E4FF1276EEE4FDFF1276A5
:102E7200EE7D04E4FF1276EE7D527F041276EE754B
:102E82005200755398D269022F5BD26BAF51125A1E
:102E9200497D577F021276EE7D05E4FF1276EEE45D
:102EA200FDFF1276EE7D05E4FF1276EE7D527F0481
:102EB2001276EE7552007553A0D269022F5BD26B67
:102EC200AF51125A497D577F021276EE7D05E4FF1B
:102ED2001276EEE4FDFF1276EE7D06E4FF1276EE48
:102EE2007D527F041276EE7552007553A8D2698026
:102EF20068D26BAF51125A497D577F021276EE7D2E
:102F020005E4FF1276EEE4FDFF1276EE7D07E4FFA4
:102F12001276EE7D527F041276EE7552007553B032
:102F2200D2698035D26BAF51125A497D577F021256
:102F320076EE7D05E4FF1276EEE4FDFF1276EE7D7D
:102F420008E4FF1276EE7D527F041276EE7552008F
:102F5200755378D2698002C269306909AF53AE52A3
:102F62001261C88005AF511279C0C26BAF51125ABB
:012F72004915
:012F7300223B
:08315E008E518F528D538B54EA
:10316600C2698F828E83A3A3E0640A6003023215CC
:10317600124AA48E568F57D3E557943BE5569400D2
:103186005003023210E5579408E5569407507BC366
:10319600E5536480948A5072855282855183A3A335
:1031A600A3E0F555B401069006000232BBE555B41E
:1031B60002069006020232BBE555B40306900604E9
:1031C6000232BBE555B404069006060232BBE5554D
:1031D600B405069006080232BBE555B4060690060D
:1031E6000A0232BBE555B4070690060C0232BBE56F
:1031F60055B4080690060E0232BBE555B409069092
:1032060006100232BBD269023337D26902333785E0
:103216005282855183A3A3E0640160030232C5ADE7
:1032260053AF52AE51124AA48E568F57D3E55794D8
:103236003BE55694005003023337E5579408E556AC
:1032460094074003023337C3E5536480948A4003EE
:10325600023337855282855183A3A3A3E0F555B483
:103266000A05900612804EE555B4010590061480B5
:1032760044E555B40205900616803AE555B40305B3
:103286009006188030E555B4040590061A8026E5A8
:1032960055B4050590061C801CE555B40605900638
:1032A6001E8012E555B407059006208008E555B442
:1032B6000809900622E556F0A3806FD269807285D0
:1032C6005282855183A3A3E064027065AD53AF5269
:1032D600AE51126B937556008F57C3E5579463E54D
:1032E600569400504CC3E5536480948850438552ED
:1032F60082855183A3A3A3E0F555B4010790063058
:10330600EFF0802DE555B40205900631801CE55599
:10331600B403059006328012E555B40405900633D1
:103326008008E555B40508900634E557F08002D2CA
:0F33360069306904C26A8002D26AAF54127B9474
:013345002265
:10267D008F518D528B53E551640A6003022729E572
:10268D0052C3940A40030228FFD26BAF53125A492A
:10269D007D277F081276EE7D06E4FF1276EEE4FDCF
:1026AD00FF1276EEAD52E4FF1276EE7D527F0412EC
:1026BD0076EEE55214B4090040030228F89026D8AE
:1026CD0075F003A4C58325F0C583730226F3022696
:1026DD00F90226FF02270502270B022711022717F1
:1026ED0002271D02272390060002283990060202B8
:1026FD0028399006040228399006060228399006DA
:10270D000802283990060A02283990060C02283949
:10271D0090060E022839900610022839E551640101
:10272D006003022847E552D394004006E552940910
:10273D004009E552640A6003022844D26BAF53127C
:10274D005A497D277F081276EE7D06E4FF1276EE5C
:10275D00E552B40A147D0AE4FF1276EE7D527F0431
:10276D001276EE900612022839E552B401147D0B53
:10277D00E4FF1276EE7D527F041276EE900614027F
:10278D002839E552B402147D0CE4FF1276EE7D5229
:10279D007F041276EE900616022839E552B4031323
:1027AD007D0DE4FF1276EE7D527F041276EE9006DB
:1027BD00188079E552B404137D0EE4FF1276EE7D98
:1027CD00527F041276EE90061A8061E552B405131D
:1027DD007D0FE4FF1276EE7D527F041276EE9006A9
:1027ED001C8049E552B406137D10E4FF1276EE7D90
:1027FD00527F041276EE90061E8031E552B4071317
:10280D007D11E4FF1276EE7D527F041276EE900676
:10281D00208019E552640860030229067D12FF121B
:10282D0076EE7D527F041276EE900622E0FEA3E056
:10283D00FF12757F0229060228FFE551640260032D
:10284D00022906E552D3940050030228FFE5529465
:10285D000740030228FFD26BAF53125A497D277FE1
:10286D00081276EE7D06E4FF1276EE7D14E4FF127B
:10287D0076EEE55224FE6020146030146040146042
:10288D0050240470667D01E4FF1276EE7D527F04C4
:10289D001276EE900630804A7D02E4FF1276EE7DD0
:1028AD00527F041276EE90063180377D03E4FF12DD
:1028BD0076EE7D527F041276EE90063280247D04F2
:1028CD00E4FF1276EE7D527F041276EE9006338091
:1028DD00117D05E4FF1276EE7D527F041276EE90A7
:1028ED000634E0FF7E001275E0800EAF531279C002
:1028FD008007C26AAF53127B94C26BAF53125A4911
:01290D0022A7
:064AA4008E588F59A90590
:104AAA007D057C00E5592DF582E5583CF583E0C388
:104ABA00940A400CE5592DF582E5583CF583E4F05B
:104ACA000DBD00010CED640A4C70D9B90610E55908
:104ADA002405F582E43558F583E0FF7E0022E96477
:104AEA00077019E5592405F582E43558F583E07510
:104AFA00F00AA4ACF0FDE55924068032E964087096
:104B0A003DE5592405F582E43558F583E075F064EE
:104B1A00A4ACF0FDE5592406F582E43558F583E0A6
:104B2A0075F00AA42DFDE5F03CFCE5592407F58251
:104B3A00E43558F583E02DFDE43CAF05FE22E96437
:104B4A0009705AE5592405F582E43558F583E0FFE2
:104B5A007E007C037DE81258FCAC06AD07E55924BB
:104B6A0006F582E43558F583E075F064A42DFDE579
:104B7A00F03CFCE5592407F582E43558F583E075E5
:104B8A00F00AA42DFDE5F03CFCE5592408F582E481
:104B9A003558F583E02DFDE43CFEAF0522E4FEFF27
:014BAA0022E8
:066B93008E588F59A90580
:106B99007F057E00E5592FF582E5583EF583E0C370
:106BA900940A400CE5592FF582E5583EF583E4F047
:106BB9000FBF00010EEF64084E70D9E96407702019
:106BC900E5592405F582E43558F583E075F00AA402
:106BD900FFE5592406F582E43558F583E02FFF22B5
:026BE9007F002B
:016BEB002287
:104BAB008F56E556D3945940147D5AE4FF1276EE96
:104BBB00E55624A6FD7003024CAC024CA7E556D378
:104BCB00944F401AE556945A50147D50E4FF1276D8
:104BDB00EEE55624B0FD7003024CAC024CA7E55633
:104BEB00D39445401AE556945050147D46E4FF1279
:104BFB0076EEE55624BAFD7003024CAC024CA7E5E9
:104C0B0056D3943B4019E556944650137D3CE4FF34
:104C1B001276EEE55624C4FD7003024CAC807DE5A4
:104C2B0056D394314016E556943C50107D32E4FF38
:104C3B001276EEE55624CEFD60678060E556D39480
:104C4B00274016E556943250107D28E4FF1276EE7D
:104C5B00E55624D8FD604A8043E556D3941D401693
:104C6B00E556942850107D1EE4FF1276EEE556248F
:104C7B00E2FD602D8026E556D394134016E556943D
:104C8B001E50107D14E4FF1276EEE55624ECFD6009
:104C9B00108009E556C394145007AD56E4FF127605
:024CAB00EE22F7
:1075E0008E548F557C007D0A12590EAD07E4FF12B0
:1075F00076EE7D5B7F061276EEAE54AF557C007D55
:107600000A12590EE4FF1276EE7D4A7F070276EEEB
:04757F008E548F5542
:107583007C007D3C12590E124BAB7D057F061276B3
:10759300EEAE54AF557C007D3C12590EED4C600CA1
:0C75A300AF05124BAB7D4A7F071276EE5D
:0175AF0022B9
:0270B0008D5100
:1070B200D3EF648094804038EF648094955031EF30
:1070C2003395E0FEEF7805C333CE33CED8F9246092
:1070D200F58274033EAF82FEE4FD0FEFAA06700153
:1070E2000E14F5828A83E4F00DBD20EED26A80028E
:0770F200C26AAF51127B944A
:0170F9002274
:107361008F51900640E0D394024015D269125AFD24
:10737100753D037F327E00127A15E53D70FC801564
:10738100D269AF51125AFD7D1B7F061276EE7D0C3C
:0D7391007F031276EEC269AF51125AFD2241
:107B62007E10900640E4F0A3DEFC7E10D26A127B07
:017B7200947E
:017B730022EF
:1078A1008F5CD26B125A497D607F021276EE7D3277
:1078B1007F061276EE7D1E7F051276EEC26BAF5CFF
:0478C100125A4922EC
:1079C0008F5CD26B125A497D607F021276EE7D3059
:0D79D0007F031276EEC26BAF5C125A4922A3
:0E7B94008F5B306A030278A1AF5B1279C022CA
:1066DF002432F58274003EF583EDF0AF55EF33951C
:1066EF00E0FEE5522FF582E5513EF583E582240465
:1066FF00F582E43583F583E0FFE555FD3395E0FC46
:10670F00E5522DF582E5513CF583E5822405F582AE
:07671F00E43583F583E0FD82
:10672600EFD394004015EF940B5010EFC3940A502A
:1067360008EF75F00AA4FE8002E4FEEDD394004053
:106746000EED940B5009EDC3940A5003ED2EFEAFE7
:01675600063C
:01675700221F
:03000000027B85FB
:0F7B8500758E0078FEE4F6D8FD75816C02518094
:107AAC00D292C0F075F008C29100A29233D291D557
:067ABC00F0F5D0F0FF22FE
:107AC200EFC0F075F00833C291929333D291D5F0A2
:067AD200F6D0F0C2912283
:1076EE00EFFEEDFF1280008E2F8F30125CFC755F67
:1076FE0064AF5F155FEFD39400400EE4F55EE55E78
:09770E00C3943A50EC055E80F5CD
:01771700224F
:105CFC00D2A885A86175A881C244853082852F837E
:105D0C00E493F560C4540FF5604360F0856080C285
:105D1C0084D28500C2870000D287007580FF758011
:105D2C00FEC284C28500C28700000000D2870075C5
:105D3C0080FFD24475623E756380E4F56030941D3B
:105D4C000560E560B464F6123346E56315637002D2
:105D5C001562D3E5639400E562940050DD75623EF4
:105D6C00756380E4F56020941D0560E560B464F60D
:105D7C00123346E563156370021562D3E563940034
:105D8C00E562940050DD8561A8C2A87F147E0012E4
:025D9C007A1576
:015D9E0022E2
:107718007580FDC284C28500C28700000000D28740
:10772800007580FF7F147E00127A157F997E0912FA
:0A77380080008E2F8F30125CFC22BF
:1058DA00C2D530F707B2D563F0FF05F030E70CB256
:1058EA00D5F4048463F0FF05F080018430D502F416
:0258FA00042286
:1058FC00EF8DF0A4A8F0CF8CF0A428CE8DF0A42EC0
:02590C00FE2279
:10590E00BC000BBE0029EF8DF084FFADF022E4CC7D
:10591E00F875F008EF2FFFEE33FEEC33FCEE9DEC46
:10592E00984005FCEE9DFE0FD5F0E9E4CEFD22ED8C
:10593E00F8F5F0EE8420D21CFEADF075F008EF2FD6
:10594E00FFED33FD4007985006D5F0F222C398FDC7
:05595E000FD5F0EA2264
:10596300EB9FF5F0EA9E42F0E99D42F0E89C45F09A
:015973002211
:105974007401FF3395E0FEFDFC080808E6CF2FF61E
:1059840018E6CE3EF618E6CD3DF618E6CC3CF622F7
:107B7400EFC39461400AEF947B5005EF24E0FF22A9
:017B840022DE
:00000001FF
